:200000000C949E000C94C6000C94C6000C94C6000C94C6000C94C6000C94C6000C94C600D8
:200020000C94C6000C94C6000C94C6000C94C6000C94C6000C94C6000C94C6000C94C60090
:200040000C94C6000C94C6000C941B300C94C6000C9425310C94C6000C94C6000C94C6005B
:200060000C94C6000C94C6000C94C6000C94C6000C944D310C94C6000C94C6007C3C3E5EAA
:200080002B3D3F2F5B5D3B2C2A225C00002124272A002225282B00202326290202020202F7
:2000A0000202020404040404040404030303030303030301010101010101010102040810DB
:2000C000204080010204081020408001020408102040808040201008040201000000010240
:2000E000000000000000000403070600000000000000000000000000000000494E46494E78
:200100004954594E414ECDCCCC3D0AD7233C17B7D13877CC2B329595E6241FB14F0A000056
:2001200020410000C84200401C4620BCBE4CCA1B0E5AAEC59D7471062F2FC93211241FBE19
:20014000CFEFD0E1DEBFCDBF15E0A0E0B1E0EAE9F6E702C005900D92AC32B107D9F71DE0F8
:20016000ACE2B5E001C01D92A630B107E1F711E0CCE3D1E004C02297FE010E941638C633D0
:20018000D107C9F70E940C350C944B3B0C94000080912E07882399F14091AD035091AE0390
:2001A0006091AF037091B00380912C0790912D072CE235E00E94B623882319F140912F07F5
:2001C000509130076091310770913207411551056105710591F080912C0790912D072CE2F4
:2001E00035E00E94B623882361F010922F0710923007109231071092320710922E0781E0D5
:20020000089580E00895EF92FF920F931F937B018C010E94C8008823A9F0ECE2F5E01192E1
:2002200087E0EC32F807D9F7E092AD03F092AE030093AF031093B00380912E078160809340
:200240002E0781E01F910F91FF90EF900895DF92EF92FF920F931F937B018C01D42E80911A
:20026000AD039091AE03A091AF03B091B0038E159F05A007B107C1F00E94C8008823D9F0F0
:2002800080912C0790912D07B801A7012CE235E00E94B024882379F0E092AD03F092AE0362
:2002A0000093AF031093B00380912E078D2980932E0781E001C080E01F910F91FF90EF907F
:2002C000DF9008958F929F92AF92BF92CF92DF92EF92FF920F931F93CF93DF936C01142F72
:2002E00070932D0760932C07442321F488249924540140C0453008F01CC160E070E080E02D
:2003000090E040E00E942701882309F412C1C12FD0E02197FE0174E0EE0FFF1F7A95E1F75B
:20032000E45DFA4FE254FE4F8081EE5BF14090E08F779070892B09F0FCC0E653FE4F8081CF
:200340009181A281B38184369105A105B10508F4F0C064E0CC0FDD1F6A95E1F7CE50D94FA4
:2003600088809980AA80BB8081149104A104B10409F4DFC0C501B40140E00E9427018823C7
:2003800009F4D7C080913705909138058050924009F0CFC020913C05222309F4CAC0809125
:2003A0003A0590913B05892B09F4C3C080913905882309F4BEC0F601228B809139058483FA
:2003C000158661E070E007C04F5FF60145874150483008F0AEC0F6014585848190E09B0178
:2003E000042E02C0220F331F0A94E2F78217930759F720914205309143052115310519F016
:2004000040E050E008C020915005309151054091520550915305F60125833683478350874D
:20042000E0903A05F0903B0500E010E0E80CF91C0A1D1B1DE38AF48A058B168B80913D05A6
:2004400090913E05918F808F60913C0570E080E090E00E9485376E0D7F1D801F911FF601FC
:20046000628F738F848F958F20913D0530913E0555E0220F331F5A95E1F721503E4F232F8C
:200480003327269540E050E0260F371F481F591F26873787408B518B80913F0590914005C0
:2004A000009719F0A0E0B0E008C080914C0590914D05A0914E05B0914F0585017401E21ADF
:2004C000F30A040B150BA8019701280F391F4A1F5B1FF601058404C05695479537952795AA
:2004E0000A94D2F72187328743875487253FFFE03F07F0E04F07F0E05F0710F48CE006C074
:20050000255F3F4F4040504028F480E1F601878B81E010C08091580590915905A0915A0585
:20052000B0915B05F601828F938FA48FB58F80E2EECF80E0DF91CF911F910F91FF90EF90CC
:20054000DF90CF90BF90AF909F908F9008954F925F926F927F928F929F92AF92BF92CF922B
:20056000DF92EF92FF920F931F93CF93DF93EC016A017B01280139014230510561057105F5
:2005800008F46FC089859A85AB85BC850196A11DB11D84179507A607B70708F462C02B89FB
:2005A0003C894D895E898F89803129F499278F2D7E2D6D2D09C0C701B60117E0969587958C
:2005C000779567951A95D1F74B015C01820E931EA41EB51E8091AD039091AE03A091AF03A7
:2005E000B091B00388169906AA06BB0639F0C501B40140E00E942701882399F18F898031CD
:2006000049F4F601F070EE0FFF1FE45DFA4F518240820DC0F601EF77F070EE0FFF1FEE0F6A
:20062000FF1FE45DFA4F408251826282738280912E07816080932E078A89823080F08D81F2
:200640009E81AF81B885880E991EAA1EBB1E80922F0790923007A0923107B092320781E039
:2006600001C080E0DF91CF911F910F91FF90EF90DF90CF90BF90AF909F908F907F906F9073
:200680005F904F900895CF92DF92EF92FF920F931F93CF93DF93EC017A018B016901898577
:2006A0009A85AB85BC850196A11DB11D84179507A607B70708F450C02B893C894D895E89A3
:2006C0008F89803129F49927812F702F6F2D09C0C801B701E7E09695879577956795EA95AA
:2006E000D1F7260F371F481F591F8091AD039091AE03A091AF03B091B003281739074A078E
:200700005B0739F0CA01B90140E00E942701882319F18F89803159F4F701F070EE0FFF1FA1
:20072000E45DFA4F80819181A0E0B0E00EC0F701EF77F070EE0FFF1FEE0FFF1FE45DFA4FC0
:2007400080819181A281B381BF70F60180839183A283B38381E001C080E0DF91CF911F9195
:200760000F91FF90EF90DF90CF900895AF92BF92CF92DF92EF92FF920F931F93DF93CF93C2
:2007800000D000D0CDB7DEB76C017A018B0182E090E0A0E0B0E0F60180839183A283B383E1
:2007A0005E010894A11CB11CC601B801A70195010E944303882319F1C601B801A70100E051
:2007C00010E020E030E00E94A7028823C1F0E980FA800B811C81F6018789803129F088EF1E
:2007E0009FEFAFEFBFE004C088EF9FEFA0E0B0E0E816F9060A071B07B8F281E001C080E0F9
:200800000F900F900F900F90CF91DF911F910F91FF90EF90DF90CF90BF90AF9008954F9254
:200820005F926F927F928F929F92AF92BF92CF92DF92EF92FF920F931F93DF93CF9300D0F5
:2008400000D0CDB7DEB76C0149835A836B837C833901EE24FF2487012E010894411C511C20
:20086000812CA2E09A2EA12CB12C49815A816B817C81C60192010E944303882351F1D50144
:20088000C401F601058404C0880F991FAA1FBB1F0A94D2F7E80EF91E0A1F1B1F29813A8121
:2008A0004B815C818789803129F088EF9FEFAFEFBFE004C088EF9FEFA0E0B0E0281739071B
:2008C0004A075B0790F2F301E082F1820283138381E00F900F900F900F90CF91DF911F91A2
:2008E0000F91FF90EF90DF90CF90BF90AF909F908F907F906F905F904F9008952F923F9295
:200900004F925F926F927F928F929F92AF92BF92CF92DF92EF92FF920F931F93DF93CF9303
:20092000CDB7DEB72F970FB6F894DEBF0FBECDBF1C014A875B876C877D873F872E87D90175
:200940000D911D912D913C91011511052105310549F0480159010894811C911CA11CB11CEC
:20096000198610C0FC0180809180A280B38019868A859B85AC85BD850197A105B10511F46B
:2009800091E09987D10119968D919D910D90BC91A02D0196A11DB11D8D839E83AF83B8877D
:2009A000750164014424552432018E010F5F1F4FF10181859285A385B485481659066A0640
:2009C0007B0608F090C08D819E81AF81B8858C159D05AE05BF0550F482E0882E912CA12C14
:2009E000B12CB2E0CB2ED12CE12CF12CC101B701A60198010E944303882309F474C08981E0
:200A00009A81AB81BC81A70196012F5F3F4F4F4F5F4F0097A105B10519F049015A010DC03D
:200A2000281939094A095B098A859B85AC85BD85281739074A075B0759F00894411C511CF9
:200A4000611C711C0894C11CD11CE11CF11CB0CFC101A601B7010FEF1FEF2FEF3FE00E9491
:200A6000A702882399F43FC02601370108944108510861087108C101B301A20197018601DF
:200A80000E94A702882379F1730162018C149D04AE04BF0448F3AE85BF854D915D916D91ED
:200AA0007C91411551056105710539F0C101950184010E94A7028823B1F0EE85FF8580820B
:200AC0009182A282B382F985FF2359F00894811C911CA11CB11CD1018D929D92AD92BC92A4
:200AE000139781E001C080E02F960FB6F894DEBF0FBECDBFCF91DF911F910F91FF90EF9090
:200B0000DF90CF90BF90AF909F908F907F906F905F904F903F902F9008958130910579F074
:200B2000823091051CF4009741F00EC08230910541F08330910541F406C05F9A05C0469A6C
:200B400003C02B9A01C0299AFC01EE0FFF1FEE0FFF1FE553F84F80819181A281B3810196D6
:200B6000A11DB11D80839183A283B3835F9846982B98299808950F931F93CF93DF938C01CC
:200B8000EB012130310519F02FEF3FEF4BC081E030C0DF01AA0FBB1FAA0FBB1FAC0FBD1F94
:200BA00012966D917C911397601771070CF53197EE0FFF1FEE0FFF1FEC0FFD1F228133817C
:200BC0000190F081E02D021B130B8D919C918E1B9F0B621B730B9C01029FC001039F900DF4
:200BE000129F900D11240E94B0376E0F7F1F16C08F5FE82FF0E0E417F5075CF2E417F507E7
:200C000019F060E070E00AC041505040440F551F440F551FC40FD51F688179812FEF33E0E7
:200C2000261B370BC901DF91CF911F910F910895CF93DF93EB012130310519F06FEF7FEF8E
:200C40004CC02FEF33E0281B390B81E031C0DF01AA0FBB1FAA0FBB1FAC0FBD1F6D917C91D6
:200C60001197261737071CF53197EE0FFF1FEE0FFF1FEC0FFD1F408151810280F381E02D95
:200C8000241B350B12968D919C9113978E1B9F0B641B750BAC01249FC001259F900D349F81
:200CA000900D11240E94B0376E0F7F1F16C08F5FE82FF0E0E417F50754F2E417F50719F0D6
:200CC00060E070E00AC041505040440F551F440F551FC40FD51F6A817B81CB01DF91CF91C1
:200CE0000895AF92BF92CF92DF92EF92FF920F931F93E0903404F0903504A0903A04B0907E
:200D00003B04C0903C04D0903D04662777276E197F09882777FD8095982F0E941736A60194
:200D200095010E947C350E94E4357093430B6093420B0027F7FC0095102FC801B7010E946D
:200D40001736A60195010E947C350E94E4357093450B6093440B04E414E085E090E0B801FC
:200D60004EE150E021E030E00E94BB059093470B8093460B8CE291E0B8014EE150E021E0D0
:200D800030E00E94BB059093490B8093480B10925B0B10925C0B10925F0B1092610B82E077
:200DA00090E0A0E0B0E08093620B9093630BA093640BB093650B1092790B84E295E0909329
:200DC000810B8093800B1092840B90939D0B80939C0B1092A00B1F910F91FF90EF90DF9019
:200DE000CF90BF90AF900895EF92FF920F931F93CF93DF930E948B302091510730915207AF
:200E00004091530750915407621B730B840B950B603771058105910508F41DC10E948B30E1
:200E20006093510770935207809353079093540787E00E943F2FCFEFD3E0C81BD90BD0930E
:200E40002B0BC0932A0B8091460B9091470B8C179D0784F082E090E09093380780933707BF
:200E600081E090E090933A07809339071092290B1092280B8091480B9091490BC817D907A7
:200E800024F01092290B1092280B0091280B1091290B0C1B1D0B1093410B0093400BB80125
:200EA000882777FD8095982F0E941736209136043091370440913804509139040E94CB368F
:200EC0000E94E4357B017093390B6093380B8091340B9091350B800F911F2091420B3091AF
:200EE000430B821793074CF04091440B5091450B9C01481759070CF49A013093350B209337
:200F0000340BB901882777FD8095982F0E94173620913A0430913B0440913C0450913D04C8
:200F20000E94CB360E94E4358B0170933B0B60933A0B8091360B9091370BBE01681B790BCB
:200F4000882777FD8095982F0E94173620913E0430913F0440914004509141040E94CB36CE
:200F60000E94E4359B0170933D0B60933C0BD093370BC093360BB701621B730B600F711FAA
:200F800077FF03C060E070E008C08091320490913304861797070CF4BC0170933F0B6093E9
:200FA0003E0B8DE00E945D2F80913707909138070297D9F02091280B3091290B8091460B01
:200FC0009091470B821793079CF480913B0790913C07019690933C0780933B07019705979E
:200FE00044F010923C0710923B0780E180B901C0149A0E948B302091550730915607409192
:20100000570750915807621B730B840B950B6858734180409040F8F00E948B306093550770
:2010200070935607809357079093580786E00E943F2F2FEF33E0281B390B30932F0B20937F
:201040002E0B80912C0B90912D0B2817390714F05A9801C05A9ADF91CF911F910F91FF90DD
:20106000EF9008958091390790913A07019741F4109238071092370710923A07109239074E
:201080000E948B3020912A0B30912B0B8091280B9091290B2817390724F410923807109263
:2010A000370708952F923F924F925F926F927F928F929F92AF92BF92CF92DF92EF92FF9217
:2010C0000F931F93DF93CF93CDB7DEB7C856D0400FB6F894DEBF0FBECDBFA3969FAF8EAF96
:2010E000A3976091AB077091AC078091AD079091AE072091BB073091BC074091BD07509157
:20110000BE070E94C736181614F4459801C0459A6091AF077091B0078091B1079091B207B6
:201120002091BF073091C0074091C1075091C2070E94C736181614F4479A01C04798609126
:20114000B3077091B4078091B5079091B6072091C3073091C4074091C5075091C6070E947A
:20116000C736181614F42A9A01C02A986091B7077091B8078091B9079091BA072091C70754
:201180003091C8074091C9075091CA070E94C736181614F4289801C0289A80913D07882354
:2011A00059F4329B09C0A396AEADBFADA3971D921D921D921C92139780913E07882351F467
:2011C000339B08C0A396EEADFFADA397148215821682178280913F07882361F4349B0AC071
:2011E000A396AEADBFADA39718961D921D921D921C921B97A396EEADFFADA397A080B1808F
:20120000C280D380A114B104C104D10409F05E98A3962EAD3FADA3972C5F3F4F3AAF29AF32
:20122000A396AEADBFADA3971496ED90FD900D911C911797E114F1040105110509F05E98D2
:20124000A396EEADFFADA3973896F8AFEFABA396AEADBFADA39718962D913D914D915C9186
:201260001B97211531054105510509F01598A396EEADFFADA3973C96A196FFAFEEAFA197C8
:20128000A396AEADBFADA3971C966D917D918D919C911F976F966CAF7DAF8EAF9FAF6F9778
:2012A000611571058105910509F05E98FE01319680E1DF011D928A95E9F7A982BA82CB82CE
:2012C000DC82ED82FE820F83188729873A874B875C876F966CAD7DAD8EAD9FAD6F976D87A1
:2012E0007E878F87988BAE14BF04C006D106B0F42E153F054007510760F46E157F058007E2
:20130000910738F481E090E061969FAF8EAF61973CC0AE14BF04C006D106A8F02A153B0589
:201320004C055D0580F46F966CAD7DAD8EAD9FAD6F976A157B058C059D0528F461961FAE9F
:201340001EAE619722C02A153B054C055D05B8F02E153F054007510790F06F968CAD9DADDF
:20136000AEADBFAD6F9782179307A407B50738F4A2E0B0E06196BFAFAEAF619706C0E3E085
:20138000F0E06196FFAFEEAF61976196EEADFFAD6197EE0FFF1FEE0FFF1FEC0FFD1F21811E
:2013A0003281438154812BAB3CAB4DAB5EAB56954795379527956B962CAF3DAF4EAF5FAF01
:2013C0006B976896BFAD68976996AFAD69976A967FAD6A976B966FAD6B9720E030E080E08B
:2013E00090E0AE014F5E5F4F6196EEADFFAD61972E173F0739F0FA01E80FF91FB083A18328
:2014000072836383FC01E553F84F10821182128213822F5F3F4F04962430310529F76196D0
:20142000EEADFFAD6197EE0FFF1FEE0FFF1FDF01A552B84F2D913D914D915C9167962CAF2A
:201440003DAF4EAF5FAF67972093A7073093A8074093A9075093AA07E759F84F7080618055
:201460003281A4963FAFA4974381A5964FAFA5977092990760929A0730939B0740939C070D
:2014800061968EAC9FAC6197272D362DA4964FADA497A5965FADA597C901DA017C018D017D
:2014A000CC24DD24AA24BB24A396EEADFFADA397EA0DFB1D2081318142815381211531056F
:2014C0004105510551F161966EAD7FAD6197C616D70619F1F501E759F84F208031804280A5
:2014E0005380C201B1010E948537F401EE0FFF1FEE0FFF1FA396AEADBFADA397EA0FFB1FCE
:2015000020813181428153810E94C337E216F3060407150710F4460102C017012801089443
:20152000C11CD11CE4E0F0E0AE0EBF1EF4E0CF16D10419F082017101B7CF60E071EE85EF8F
:2015400095E0272D362DA4964FADA497A5965FADA5970E94C337C901DA0127968CAF9DAFE6
:20156000AEAFBFAF27979401220F331F220F331FA3964EAD5FADA397420F531F5AAB49AB11
:201580001EAE1DAE1CAE1BAEA396EEADFFADA3976BAD7CADE60FF71F608071808280938035
:2015A000611471048104910409F44FC0C201B1010E9415365B016C01A9A9BAA96D917D912F
:2015C0008D919C910E9415367B018C01C401B3010E9415369B01AC01C801B7010E947C3547
:2015E0009B01AC01C601B5010E94CB360E94E9359B01AC01E1E2F0E0EC0FFD1F6BAD7CAD8E
:20160000E60FF71F20833183428353838DAD9EAD6196AEADBFAD61978A179B07B1F42093F7
:20162000990730939A0740939B0750939C0760E071EE85EF95E00E94C337C901DA01279625
:201640008CAF9DAFAEAFBFAF2797EDADFEAD3196FEAFEDAF2BAD3CAD2C5F3F4F3CAF2BAF86
:20166000349709F091CF2BED422E27E0522E91E2692E712C6C0E7D1EA8961FAEA897A996F2
:201680001FAEA99722243324CC24DD24A396EEADFFADA397EC0DFD1D80819181A281B38178
:2016A0000097A105B10509F47DC06F964CAD5DAD6EAD7FAD6F97411551056105710561F1CE
:2016C000D2016D917D918D919C910E9417369B01AC0160E27CEB8EEB9CE40E947C357B0137
:2016E0008C01F30160817181828193810E9415369B01AC0160E27CEB8EEB9CEC0E947C354C
:201700009B01AC01C801B7010E9414357B018C01F601E758F84F2BC0D2016D917D918D91A6
:201720009C910E9417369B01AC0160E27CEB8EEB9CE40E947C357B018C01F301608171817F
:20174000828193810E9415369B01AC0160E27CEB8EEB9CEC0E947C359B01AC01C801B70175
:201760000E9414357B018C01F601E757F84F60817181828193810E9415369B01AC01C80110
:20178000B7010E947C354B015C01A8966FADA897A9967FADA997C101A50194010E94C736B5
:2017A00018164CF4A8968FADA897A9969FADA997D1014C015D0124E030E0C20ED31E420E95
:2017C000531E620E731E30E1C316D10451F0D501C401A8968FAEA897A9969FAFA9971D0157
:2017E00055CF61960EAD1FAD6197000F111F000F111FF801E552F84F608171818281938170
:201800000E9417369B01AC0160E27CEB8EEB9CE40E947C356B017C010C0F1D1FD80191965B
:201820006D917D918D919C9194970E9415369B01AC0160E27CEB8EEB9CEC0E947C359B0157
:20184000AC01C701B6010E941435A50194010E947C350E94E93560939D0770939E078093D1
:201860009F079093A0070E94153620E030E040E05FE30E94CB36A50194010E94CB367B019C
:201880008C0127966CAD7DAD8EAD9FAD27970E9417369B01AC01C801B7010E941435A5012C
:2018A00094010E94CB360E94E4350E9415362EEA37E441E85FE30E94CB360E94E935609354
:2018C000A1077093A2078093A3079093A40781E08093A5078091990790919A07A0919B07C3
:2018E000B0919C0767962CAD3DAD4EAD5FAD679782179307A407B50710F41092A5070E94B1
:20190000993023966CAF7DAF8EAF9FAF239724E630E040E050E00E948537609341077093B3
:201920004207809343079093440760934507709346078093470790934807609349077093EB
:201940004A0780934B0790934C0760934D0770934E0780934F079093500760E071EE85EFC6
:2019600095E067962CAD3DAD4EAD5FAD67970E94C337C901DA012B968CAF9DAFAEAFBFAFD9
:201980002B9761968EAD9FAD6197880F991F880F991FA3964EAD5FADA397480F591F63962F
:2019A0005FAF4EAF63972BA93CA94DA95EA92F962CAF3DAF4EAF5FAF2F9722243324210150
:2019C000AC014F5B584FA7965FAF4EAFA797BCC20E94F4068091A507882309F423C12114EB
:2019E00031044104510489F48091990790919A07A0919B07B0919C078093A7079093A807DE
:201A0000A093A907B093AA071DC18091A1079091A207A091A307B091A40782159305A405EF
:201A2000B50508F488C060919D0770919E0780919F079091A00720E137E240E050E00E94E2
:201A4000E537122F032FF42EE52E0E94993023962CAD3DAD4EAD5FAD2397621B730B840B90
:201A6000950B24E630E040E050E00E94C337CA01B901212F302F4F2D5E2D0E9485379B018B
:201A8000AC0127966CAD7DAD8EAD9FAD2797260F371F481F591F60E071EE85EF95E00E94C0
:201AA000E537C901DA018093A7079093A807A093A907B093AA0767962CAD3DAD4EAD5FAD34
:201AC000679782179307A407B50750F41092A6072093A7073093A8074093A9075093AA07F1
:201AE0006B964CAD5DAD6EAD7FAD6B97241635064606570608F4A6C02092A1073092A20754
:201B00004092A3075092A4072091A7073091A8074091A9075091AA0760E071EE85EF95E052
:201B20000E94C337C901DA012B968CAF9DAFAEAFBFAF2B9785C02F962CAD3DAD4EAD5FADBB
:201B40002F9782179307A407B50708F46BC08091A607882359F40E94993023966CAF7DAFDD
:201B60008EAF9FAF239731E03093A60760919D0770919E0780919F079091A00720E137E2CB
:201B800040E050E00E94E537122F032FF42EE52E0E94993023962CAD3DAD4EAD5FAD2397E7
:201BA000621B730B840B950B24E630E040E050E00E94C337CA01B901212F302F4F2D5E2DBA
:201BC0000E9485372B962CAD3DAD4EAD5FAD2B97261B370B480B590B60E071EE85EF95E098
:201BE0000E94E537C901DA018093A7079093A807A093A907B093AA072091990730919A0765
:201C000040919B0750919C07281739074A075B07C8F42093A7073093A8074093A9075093A6
:201C2000AA0710C067964CAD5DAD6EAD7FAD67974093A7075093A8076093A9077093AA0774
:201C40001092A6076396EEADFFAD639780819181A281B3810097A105B10509F475C180915A
:201C60003D078823C9F4329B17C061962EAD3FAD6197232B09F495C1A396EEADFFADA39703
:201C800080819181A281B3810097A105B10521F0108211821282138280913E078823B9F4DA
:201CA000339B15C06196EEADFFAD6197319709F478C1E9ADFAAD80819181A281B38100970F
:201CC000A105B10521F0108211821282138280913F078823B9F4349B15C06196EEADFFADB8
:201CE0006197329709F45DC1EFA9F8AD80819181A281B3810097A105B10521F01082118238
:201D0000128213820E94993024E630E040E050E00E948537A796EEADFFADA7972081318152
:201D200042815381621B730B840B950B6093FC077093FD078093FE079093FF0797FFE2C06C
:201D40000E94993024E630E040E050E00E948537A796AEADBFADA7976D937D938D939C93AF
:201D600013978091A7079091A807A091A907B091AA07B695A795979587958093FC0790934F
:201D8000FD07A093FE07B093FF07BCC00197A109B1096396EEADFFAD639780839183A283D0
:201DA000B3838091FC079091FD07A091FE07B091FF072091A7073091A8074091A907509106
:201DC000AA07821B930BA40BB50B8093FC079093FD07A093FE07B093FF0761968EAD9FAD6C
:201DE00061970E948D05A796EEADFFADA79780819181A281B3812091A7073091A8074091EB
:201E0000A9075091AA07820F931FA41FB51F80839183A283B383A3968EAC9FACA397B1E1AA
:201E2000AB2EB12CAC0EBD1E3E010894611C711CCC24DD2461962EAD3FAD6197C216D3061A
:201E4000E1F1F40180819181A281B3810097A105B10599F1D501ED90FD900D911C91F301B5
:201E600080819181A281B381E81AF90A0A0B1B0BD501ED92FD920D931C93139717FF1DC0E8
:201E8000C6010E948D05F40180819181A281B3810197A109B10980839183A283B3832BA9A6
:201EA0003CA94DA95EA9E20EF31E041F151FD501ED92FD920D931C9313970894C11CD11CA5
:201EC000E4E0F0E08E0E9F1EAE0EBF1E6E0E7F1EF4E0CF16D10409F0ADCF0894211C311C3A
:201EE000411C511C2F962CAD3DAD4EAD5FAD2F9721503040404050402F962CAF3DAF4EAF49
:201F00005FAF2F972091FC073091FD074091FE075091FF078091A7079091A807A091A90747
:201F2000B091AA07281739074A075B0768F06396EEADFFAD639780819181A281B3810097EA
:201F4000A105B10509F022CFE9ADFAAD80819181A281B381EFA9F8AD20813181428153816D
:201F6000820F931FA41FB51FA396EEADFFADA3972081318142815381820F931FA41FB51F09
:201F8000A196EEADFFADA1972081318142815381820F931FA41FB51F0097A105B10509F0DB
:201FA00017CD159AABEA6A2EA7E07A2EFBEBCF2EF7E0DF2EEBEC8E2EE7E09E2E71EBA72E14
:201FC00073E0B72ED601ED90FD900D911C91F3016081718182819381A80197010E94C736DF
:201FE0001816DCF4D4016D917D918D919C910E941536F50120813181428153810E947C3597
:202000009B01AC01C801B7010E941435D6016D937D938D939C93139719C0F401608171818A
:20202000828193810E941536D5012D913D914D915C910E947C359B01AC01C801B7010E94B0
:202040001335F601608371838283938324E030E0620E731EC20ED31E820E931EA20EB31EB7
:202060003BEB631637E0730609F0ACCFC859DF4F0FB6F894DEBF0FBECDBFCF91DF911F91A7
:202080000F91FF90EF90DF90CF90BF90AF909F908F907F906F905F904F903F902F900895E1
:2020A0002F923F924F925F926F927F928F929F92AF92BF92CF92DF92EF92FF920F931F938E
:2020C000DF93CF93CDB7DEB766970FB6F894DEBF0FBECDBFBDE3EB2EB7E0FB2E00E010E086
:2020E000DD24D394F801E555F84FD801A554B84F60817181828193812D913D914D915C91E4
:202100000E94C73688231CF0F701D08202C0F70110820C5F1F4F0894E11CF11C003111050D
:2021200009F76091AB077091AC078091AD079091AE0720E030E046E153E40E94C736181672
:2021400064F480E090E0A6E1B3E48093AB079093AC07A093AD07B093AE076091AF07709117
:20216000B0078091B1079091B20720E030E044E153E40E94C736181664F480E090E0A4E11F
:20218000B3E48093AF079093B007A093B107B093B2076091B3077091B4078091B5079091C9
:2021A000B60720E030E048EC52E40E94C736181664F480E090E0A8ECB2E48093B3079093D9
:2021C000B407A093B507B093B607AA24BB24F501E555F84FD501A554B84F60817181828185
:2021E00093812D913D914D915C910E9413356B017C01F501EC5FF74F608371838283938328
:2022000020E030E040E050E00E94C736181624F0F7FAF094F7F8F0948501075A184FF50151
:20222000EF54FC4FC701B60120813181428153810E94CB360E94E935F8016083718382836F
:20224000938384E090E0A80EB91E90E1A916B10409F0BDCF8091CD049091CE040A9734F4FF
:202260008AE090E09093CE048093CD04A0900408B0900508C0900608D0900708C601B501D8
:2022800020E030E040E050E00E94C736181654F0C601B50120E030E040E050E00E947835A1
:2022A0008823BCF5609108087091090880910A0890910B0820E030E040E050E00E947835A9
:2022C000882339F560910C0870910D0880910E0890910F0820E030E040E050E00E947835FC
:2022E0008823B9F4C601B50120E030E040E050E00E94C736181624F0D7FAD094D7F8D09460
:20230000A0920008B0920108C0920208D092030810C1C601B50120E030E040E050E00E941F
:202320007835882309F060C0E0900808F090090800910A0810910B08C801B70120E030E033
:2023400040E050E00E94C736181654F0C801B70120E030E040E050E00E9478358823E4F469
:2023600060910C0870910D0880910E0890910F0820E030E040E050E00E947835882361F434
:20238000C801B70120E030E040E050E00E94C73618160CF4C6C0C1C0C801B70120E030E0F7
:2023A00040E050E00E9478358823F1F4E0900C08F0900D0800910E0810910F08C801B701F5
:2023C00020E030E040E050E00E94C73618160CF4A8C0C801B70120E030E040E050E00E94E5
:2023E000783588230CF499C0C601B50120E030E040E050E00E94C73618163CF1C601B501D8
:2024000020E030E040E050E00E94783587FD1DC0E0900808F090090800910A0810910B0844
:20242000C801B70120E030E040E050E00E94C73618165CF0C801B70120E030E040E050E0C1
:202440000E94783588230CF04BC0E0900808F090090800910A0810910B08C601B501A601EF
:2024600095010E94CB365B016C01C801B701A80197010E94CB369B01AC01C601B5010E948D
:2024800014350E9432377B018C01A0900C08B0900D08C0900E08D0900F08C601B50120E0EC
:2024A00030E040E050E00E94C7361816D4F5C801B701A80197010E94CB367B018C01C601F1
:2024C000B501A60195010E94CB369B01AC01C801B7010E9414350E9432377B018C0121C0BC
:2024E000E0901008F09011080091120810911308C801B70120E030E040E050E00E94C736D4
:2025000018167CF0C801B70120E030E040E050E00E94783588230CF010C117FB109517F9B2
:202520001095E0920008F092010800930208109303086091CD047091CE04882777FD8095D9
:20254000982F0E94173620EC31EE44E65CE40E947C359B01AC016091000870910108809180
:202560000208909103080E947C353B014C011A8A198AE989FA89E75AF84F80819181A2814F
:20258000B3810097A105B10509F463C0E989FA89EC5FF74FA080B180C280D380C601B5010B
:2025A00020E030E040E050E00E94C73618161CF48601750106C08601750117FB109517F957
:2025C0001095C401B30120EC31EE44E65CE40E947C356B8B7C8B8D8B9E8BE989FA89EF5380
:2025E000FC4F2080318042805380C801B7012B893C894D895E890E947C35A20191010E94C9
:20260000C736181634F5C601B50120E030E040E050E00E94C736181624F0D7FAD094D7F8A4
:20262000D094C401B301A20191010E947C357B018C01C601B5012B893C894D895E890E94D7
:202640007C359B01AC01C801B7010E94CB363B014C01E989FA893496FA8BE98B709709F01B
:2026600088CFC301D4018093EF079093F007A093F107B093F207EE24FF24F701E75AF84F2B
:2026800060817181828193816115710581059105C1F087010552184F0E9415369B01AC011B
:2026A000C401B3010E947C3520E030E048EC52E40E94CB360E94E435F801608371838283A1
:2026C000938384E090E0E80EF91E90E1E916F104A1F68091590790915A07A0915B07B09140
:2026E0005C0789839A83AB83BC8380915D0790915E07A0915F07B09160078D839E83AF8344
:20270000B8878091610790916207A0916307B091640789879A87AB87BC87809165079091EC
:202720006607A0916707B09168078D879E87AF87B88BCE0101960E94520866960FB6F8947C
:20274000DEBF0FBECDBFCF91DF911F910F91FF90EF90DF90CF90BF90AF909F908F907F909C
:202760006F905F904F903F902F9008950E948B3060934A0B70934B0B80934C0B90934D0B7E
:202780008091370790913807029759F587EC9BE00E942B2F60E071E00E94453387EC9BE020
:2027A0000E942B2F6091390770913A070E94663487EC9BE00E942B2F64E071E00E944533D5
:2027C00087EC9BE00E942B2FE0913907F0913A07EE0FFF1FEE53FB4F608171810E94453309
:2027E00009C0E0911C0BF0911D0BEC5EF44F8081882341F487EC9BE00E942B2F67E071E0DF
:202800000E94743308950F931F9307EC1BE0C8010E942B2F0E94AA32C8010E942B2F6AE03E
:2028200071E00E944533C8010E942B2F4091F7075091F8076091F9077091FA074F5F5F4F6A
:202840006F4F7F4F0E9453340E94B6131F910F91089540911C0B50911D0B20E630E0B9019A
:20286000469F9001479F300D569F300D1124682F772767FD7095C9018C5E974F0E94D63A6E
:202880009C019093270B8093260B80E0232B09F081E008958091260B9091270B019660E0F1
:2028A00070E00E941A3808951092C10B8091840B882321F080E89BE00E94DE2686E59BE0FE
:2028C00060E04FE10E94C024882339F487EC9BE00E942B2F62E171E027C082E69BE066E597
:2028E0007BE041E00E946201882381F482E69BE066E57BE040E00E946201882339F487EC3E
:202900009BE00E942B2F6FE171E00EC080E89BE062E67BE00E94D629882349F487EC9BE0D4
:202920000E942B2F62E371E00E947433089581E08093C10B0895AF92BF92CF92DF92EF925D
:20294000FF920F931F93CF93DF9387E40E942914882309F4CFC20E944A140E94E4356C31E3
:20296000710509F4CFC06D3171056CF477FF02C00C94531E62307105A4F06430710511F0F1
:202980000C94531E8BC06B35710509F497C26C35710509F497C26A35710511F00C94531EDB
:2029A0008AC2EBEBEE2EE7E0FE2E0BEA17E0C0E0D0E0FE01E853FB4F80810E94291488239B
:2029C00041F10E944A145B016C01FE01ED5CF84F8081882311F061E002C06091FB0770E07A
:2029E000882777FD8095982F0E941736F70120813181428153810E94CB369B01AC01C60154
:202A0000B5010E941435F80160837183828393830AC0F70180819181A281B381F801808302
:202A20009183A283B383219644E050E0E40EF51E0C5F1F4FC430D10509F0BBCF86E40E94E5
:202A400029148823E9F00E944A140E94E4357B018C017093EC076093EB07B701882777FD3B
:202A60008095982F0E94173620E030E040E050E00E94C736181624F4F092CE04E092CD04AF
:202A80000E9450100E948B3060934A0B70934B0B80934C0B90934D0B0C94551E80E50E9437
:202AA0002914882321F4AA24BB24650106C00E944A140E94E9355B016C0183E50E94291470
:202AC000882361F00E944A1420E030E04AE754E40E94CB360E94E9355B016C010E948B30F8
:202AE0007B018C01EA0CFB1C0C1D1D1D02C00E94F4060E948B306E157F0580079107B8F3D1
:202B00000C94531E8091CD049091CE049093EE078093ED078091BB079091BC07A091BD0704
:202B2000B091BE078093AB079093AC07A093AD07B093AE078091BF079091C007A091C1075D
:202B4000B091C2078093AF079093B007A093B107B093B2078091C3079091C407A091C5071D
:202B6000B091C6078093B3079093B407A093B507B093B6078091C7079091C807A091C907DD
:202B8000B091CA078093B7079093B807A093B907B093BA071092CE041092CD048091C804B5
:202BA0000E942914882371F48091C9040E942914882341F48091CA040E942914882311F41B
:202BC00081E001C080E08093CC04882339F48091C8040E942914882309F466C00F2EF0E021
:202BE000EF2EF0E0FF2EF0E00F2FF0E01F2FF02DE092BB07F092BC070093BD071093BE073A
:202C000080E090E0A1E6B3EC8093AB079093AC07A093AD07B093AE076091D1037091D203A9
:202C20008091D3039091D4030E94E4357093CE046093CD040E945010E092BB07F092BC07E6
:202C40000093BD071093BE0780E090E0A0EAB0E48093AB079093AC07A093AD07B093AE074D
:202C60000E94501080E090E0A0E2B1EC8093AB079093AC07A093AD07B093AE070E945010E7
:202C8000E092BB07F092BC070093BD071093BE07E092AB07F092AC070093AD071093AE0704
:202CA0001092CE041092CD048091CC04882339F48091C9040E942914882309F466C00F2EAC
:202CC000F0E0EF2EF0E0FF2EF0E00F2FF0E01F2FF02DE092BF07F092C0070093C107109342
:202CE000C20780E090E0AEE5B3EC8093AF079093B007A093B107B093B2076091D5037091B5
:202D0000D6038091D7039091D8030E94E4357093CE046093CD040E945010E092BF07F092E3
:202D2000C0070093C1071093C20780E090E0A0EAB0E48093AF079093B007A093B107B09346
:202D4000B2070E94501080E090E0A0E2B1EC8093AF079093B007A093B107B093B2070E949D
:202D60005010E092BF07F092C0070093C1071093C207E092AF07F092B0070093B10710935C
:202D8000B2071092CE041092CD048091CC04882339F48091CA040E942914882309F478C03C
:202DA0000F2EF0E0EF2EF0E0FF2EF0E00F2FF0E01F2FF02DE092C307F092C4070093C507BB
:202DC0001093C60780E090E0A6E1B3EC8093B3079093B407A093B507B093B6076091D90326
:202DE0007091DA038091DB039091DC030E94E4357093CE046093CD040E945010E092C30774
:202E0000F092C4070093C5071093C60780E090E0A0E0B0E48093B3079093B407A093B50718
:202E2000B093B6070E94501080E090E0A0E2B1EC8093B3079093B407A093B507B093B60707
:202E40000E94501089EC9BE060E070E00E943B2F282F30E0C901880F892F881F990B892B65
:202E600011F020503140B901882777FD8095982F0E94173620E030E048EC52E40E947C35FB
:202E80006093C3077093C4078093C5079093C6078091ED079091EE079093CE048093CD04E4
:202EA0000E948B3060934A0B70934B0B80934C0B90934D0BF8C61092FB07F5C681E080939E
:202EC000FB07F1C6C8ECD4E00BEB17E088810E942914882339F00E944A14F8016083718358
:202EE0008283938321960C5F1F4FF4E0CC3CDF0769F7D9C68DE40E942914882309F4B6C6F2
:202F00000E944A140E94E4356C35710509F44DC46D3571050CF045C06931710509F48FC15B
:202F20006A317105ECF46531710509F4FCC0663171056CF46530710509F4D7C064317105C4
:202F400009F4DCC06430710509F0ADC674C06731710509F4F2C0683171050CF067C1E8C096
:202F60006235710509F4E7C3633571056CF46B31710509F491C16B3171050CF468C16C31F6
:202F8000710509F090C6C0C16435710509F4DAC3643571050CF4D2C36535710509F083C64C
:202FA000EEC36737710509F4A8C4683771050CF56B36710509F4B8C36C3671056CF4693627
:202FC000710509F453C26A3671050CF083C36836710509F068C612C26237710509F434C4FE
:202FE0006337710509F421C46D36710509F05BC6CBC26A3C710509F4F1C46B3C71056CF4D4
:203000006E3B710509F4ECC2693C710509F4BBC46C38710509F047C610C26D3C710509F441
:203020006AC221E06D32720709F41DC56B3C710509F039C6FEC487EC9BE00E942B2F62E465
:2030400071E00E94453387EC9BE00E942B2F60913707709138070E945E3487EC9BE00E94E8
:203060002B2F64E071E00E94453387EC9BE00E942B2FE0913707F0913807EE0FFF1FE4549B
:20308000FB4F608171810E9474338091370790913807029709F007C687EC9BE00E942B2FD2
:2030A00060E071E00E94453387EC9BE00E942B2F6091390770913A070E945E3487EC9BE0E6
:2030C0000E942B2F64E071E00E94453387EC9BE00E942B2FE0913907F0913A07EE0FFF1FCD
:2030E000EE53FB4F60817181DCC5109238071092370710923A0710923907D5C587EC9BE0C3
:203100000E942B2F65E471E00E94743380E89BE060E040E00E94D52A87EC9BE00E942B2F02
:2031200065E571E0BEC51092C00B0E945414BBC51092C00B1092C10BB6C58091C10B88239C
:2031400009F4B1C51092C00B8CE99BE00E94DE268091260B9091270B04966AE270E00E948C
:20316000D63AFC01009711F0319710824091260B5091270B4C5F5F4F8CE99BE060E87BE04F
:2031800021E00E94242E882309F449C087EC9BE00E942B2F63E671E00E94453387EC9BE0FD
:2031A0000E942B2F6091260B7091270B6C5F7F4F0E94453387EC9BE00E942B2F60E771E089
:2031C0000E94453387EC9BE00E942B2F4091AE0B5091AF0B6091B00B7091B10B0E941B346C
:2031E0001092BC0B1092BD0B1092BE0B1092BF0B8091AE0B9091AF0BA091B00BB091B10B97
:203200008093B80B9093B90BA093BA0BB093BB0B87EC9BE00E942B2F67E771E042C587ECED
:203220009BE00E942B2F65E871E03BC58091C10B882309F438C581E08093C00B34C58091AE
:20324000C00B882309F42FC51092C00B2CC58091C10B882309F427C583E50E942914882346
:2032600009F421C58091260B9091270B019660E070E04AE050E00E947A39AB01BC014093C4
:20328000BC0B5093BD0B8093BE0B7093BF0B8CE99BE00E94D02507C58091C10B882369F1DE
:2032A00087EC9BE00E942B2F66E971E00E94453387EC9BE00E942B2F4091BC0B5091BD0B3F
:2032C0006091BE0B7091BF0B0E94173487EC9BE00E942B2F68EA71E00E94453387EC9BE0E7
:2032E0000E942B2F4091B80B5091B90B6091BA0B7091BB0B0E941B34D6C487EC9BE00E9401
:203300002B2F6AEA71E0CDC48091C10B882309F4CAC48CE99BE00E94DE261092C00B8091F6
:20332000260B9091270B04966AE270E00E94D63AEC01009709F120911C0B30911D0B80E67C
:2033400090E0AC01249FC001259F900D349F900D11248C5E974F6EE470E00E94D63A60E260
:2033600070E00E94D63A9C012F5F3F4F3093270B2093260B219718824091260B5091270B52
:203380004C5F5F4F8CE99BE060E87BE026E50E94242E8823E9F487EC9BE00E942B2F6AEB7B
:2033A00071E00E94453387EC9BE00E942B2F6091260B7091270B6C5F7F4F0E94453387EC3D
:2033C0009BE00E942B2F6EEC71E00E9445336BC481E08093C20B87EC9BE00E942B2F60ED0A
:2033E00071E00E94453387EC9BE00E942B2F6091260B7091270B6C5F7F4F53C483E50E9469
:203400002914882391F00E944A140E94E435DC01CB0164E474E04EE150E021E030E00E9431
:20342000BB059093290B8093280B8091390790913A07019709F037C4D0C083E50E94291419
:20344000882309F430C40E944A140E94E435DC01CB0160ED74E044E150E021E030E00E94C3
:20346000BB0590932D0B80932C0B1DC480912A0B90912B0B64E474E04EE150E021E030E05D
:203480000E9418069093310B8093300B80912E0B90912F0B60ED74E044E150E021E030E013
:2034A0000E9418069093330B8093320B87EC9BE00E942B2F62EE71E00E94453387EC9BE008
:2034C0000E942B2F6091300B7091310B0E945E3487EC9BE00E942B2F68EE71E00E944533A8
:2034E00087EC9BE00E942B2F6091320B7091330B0E946634DAC387EC9BE00E942B2F6CEE58
:2035000071E00E94453387EC9BE00E942B2F60913E0B70913F0B0E945E3487EC9BE00E940D
:203520002B2F62EF71E00E94453387EC9BE00E942B2F6091380B7091390B0E945E3487EC6B
:203540009BE00E942B2F67EF71E00E94453387EC9BE00E942B2F60913A0B70913B0B0E942A
:203560005E3487EC9BE00E942B2F6CEF71E00E94453387EC9BE00E942B2F60913C0B7091E6
:203580003D0B0E945E3491C383E50E942914882321F10E944A147B018C0160914204709116
:2035A0004304882777FD8095982F0E9417369B01AC01C801B7010E9413350E94E435DC018A
:2035C000CB0164E474E04EE150E021E030E00E94BB059093290B8093280B0E94320863C312
:2035E00083E50E942914882391F00E944A140E94E435DC01CB0164E474E04EE150E021E0F8
:2036000030E00E94BB0590932D0B80932C0B0E948B307B018C0151C00E948B306E197F09B0
:20362000800B910B695E73408040904008F443C080912A0B90912B0B64E474E04EE150E0C2
:2036400021E030E00E9418069093310B8093300B87EC9BE00E942B2F61E072E00E94453355
:2036600087EC9BE00E942B2F6091300B7091310B0E945E3487EC9BE00E942B2F68EE71E032
:203680000E94453387EC9BE00E942B2F8C0180912E0B90912F0B64E474E04EE150E021E0F8
:2036A00030E00E941806BC01C8010E9466340E948B307B018C010E94F40620912E0B3091CB
:2036C0002F0B80912C0B90912D0B281739070CF4A3CFE9C283E50E942914882319F15C9A81
:2036E0000E944A1420E030E040E050E00E94783588231CF460E070E011C00E944A1420E0FF
:2037000030E04FE753E40E94C73618161CF46FEF70E004C00E944A140E94E4358CE00E9414
:203720005D2FC1C25C9ABFC28CE060E070E00E945D2F5C98B8C210923607B5C281E08093A1
:203740003607B1C283E50E942914882399F00E944A1420E030E04AE754E40E94CB360E9480
:20376000E9356093520B7093530B8093540B9093550B99C25E9A5E9A159A5E9A94C283E5D5
:203780000E9429140E944A1420E030E04AE754E40E94CB360E94E93560934E0B70934F0BC5
:2037A0008093500B9093510B7EC2C8ECD4E001EB13E088810E942914882339F00E944A14D9
:2037C000F801608371838283938321960C5F1F4FF4E0CC3CDF0769F7C0E0D0E08E0107590D
:2037E000184FFE01E352FC4FDE01AF54BC4F60817181828193812D913D914D915C910E9413
:20380000CB369B01AC0160E27CEB8EEB9CE40E947C350E94E935F8016083718382839383BE
:203820002496C031D105D1F63EC287EC9BE00E942B2F64E072E00E94453387EC9BE00E9416
:203840002B2F6DE074E02DC287EC9BE00E942B2F6CE172E00E94453387EC9BE00E942B2FF1
:203860004091BB075091BC076091BD077091BE070E94FD3487EC9BE00E942B2F6FE172E037
:203880000E94453387EC9BE00E942B2F4091BF075091C0076091C1077091C2070E94FD348F
:2038A00087EC9BE00E942B2F62E272E00E94453387EC9BE00E942B2F4091C3075091C4073D
:2038C0006091C5077091C6070E94FD3487EC9BE00E942B2F65E272E00E94453387EC9BE0FF
:2038E0000E942B2F4091C7075091C8076091C9077091CA070E940135D6C187EC9BE00E94EB
:203900002B2F68E272E00E94453387EC9BE00E942B2F329903C06FE272E002C062E372E023
:203920000E94453387EC9BE00E942B2F65E372E00E94453387EC9BE00E942B2F339903C056
:203940006FE272E002C062E372E00E94453387EC9BE00E942B2F6CE372E00E94453387EC39
:203960009BE00E942B2F349903C06FE272E002C062E372E00E94453387EC9BE00E942B2F40
:2039800063E472E08EC148ECE42E44E0F42EC0E0D0E0F70180810E9429148823A9F00E94A5
:2039A0004A148E010758184FFE01EF54FC4F20813181428153810E94CB360E94E935F80181
:2039C00060837183828393830894E11CF11C2496FCECEF16F4E0FF06E1F665C138ECE32E9D
:2039E00034E0F32EC0E0D0E0F70180810E9429148823A9F00E944A148E010757184FFE01D3
:203A0000EF54FC4F20813181428153810E94CB360E94E935F8016083718382839383089444
:203A2000E11CF11C2496FCECEF16F4E0FF06E1F63AC18AE50E942914882309F434C10E949D
:203A40004A1420E030E048EC52E40E94CB360E94E9359B01AC0189EC9BE060E070E0422FF1
:203A60000E94362F20C180E50E942914882351F00E944A1460933604709337048093380474
:203A80009093390489E40E942914882351F00E944A1460933A0470933B0480933C049093A5
:203AA0003D0484E40E942914882351F00E944A1460933E0470933F04809340049093410458
:203AC00086E40E942914882341F00E944A140E94E43570933304609332048AE50E94291455
:203AE000882341F00E944A140E94E435709343046093420487E50E942914882341F00E94E3
:203B00004A140E94E435709335046093340487EC9BE00E942B2F64E472E00E94453387EC14
:203B20009BE00E942B2F409136045091370460913804709139040E94013587EC9BE00E9414
:203B40002B2F68E472E00E94453387EC9BE00E942B2F40913A0450913B0460913C04709108
:203B60003D040E94013587EC9BE00E942B2F6CE472E00E94453387EC9BE00E942B2F4091CB
:203B80003E0450913F0460914004709141040E94013587EC9BE00E942B2F60E572E00E9449
:203BA000453387EC9BE00E942B2F60913204709133040E94663487EC9BE00E942B2F69E5D0
:203BC00072E00E94453387EC9BE00E942B2F60913404709135040E94663487EC9BE00E9460
:203BE0002B2F64E672E00E94453387EC9BE00E942B2F60914204709143040E946634E090A0
:203C00003404F0903504662777276E197F09882777FD8095982F0E94173620913A043091DB
:203C20003B0440913C0450913D040E947C350E94E4357093430B6093420B0027F7FC0095C4
:203C4000102FC801B7010E94173620913A0430913B0440913C0450913D040E947C350E949E
:203C6000E4357093450B6093440B1DC087EC9BE00E942B2F6BE672E00E94743387EC9BE0F5
:203C80000E942B2F40911C0B50911D0B20E630E0429FB001439F700D529F700D11246C5EB3
:203CA000774F0E9474330E94B613DF91CF911F910F91FF90EF90DF90CF90BF90AF90089563
:203CC000AF92BF92CF92DF92EF92FF920F931F93DF93CF930F92CDB7DEB78091200B90912F
:203CE000210B03970CF47AC16CC24D3051F04A3341F02091230B3091240B2F3531050CF4C0
:203D00004EC1E091230BF091240B309709F459C2A0911E0BB0911F0BAC9D7001AD9DF00CA1
:203D2000BC9DF00C1124EE0DFF1DEC5EF74F10828091250B882309F02BC1AC5EB44F1C9234
:203D400087010C5E174FC8016EE470E00E94D63A9C01009709F4B0C09093270B8093260BB4
:203D60002F5F3F4F201B310B2E0D3F1DC9018C5E974F60E070E04AE050E00E947A3960934D
:203D8000F3077093F4078093F5079093F6072091F7073091F8074091F9075091FA072F5F4C
:203DA0003F4F4F4F5F4F6217730784079507D9F080911E0B90911F0B9C012C9DC0012D9DD0
:203DC000900D3C9D900D11248C5E974F6CE772E00E94E13A009739F487EC9BE00E942B2FBB
:203DE00061E872E03AC080911E0B90911F0B8C9D80018D9D100D9C9D100D1124C8018C5E7A
:203E0000974F6AE270E00E94D63A9C010097E1F140E0FF24C80102C0FE264F5FFC01E40FD8
:203E2000F11DEC5EF74FE081EA32B1F73093270B2093260BC901019660E070E00E941A3801
:203E40000E94E4352F2D30E02617370721F187EC9BE00E942B2F61EC72E00E94453387EC98
:203E60009BE00E942B2F4091F7075091F8076091F9077091FA070E9453340E9403141092A5
:203E8000240B1092230B9DC187EC9BE00E942B2F66EE72E0E2CF8091F3079091F407A0912C
:203EA000F507B091F6078093F7079093F807A093F907B093FA071EC0C8016AE270E00E9439
:203EC000D63A0097B9F087EC9BE00E942B2F66E173E00E94453387EC9BE00E942B2F409139
:203EE000F7075091F8076091F9077091FA070E945334C5CF80911E0B90911F0B8C9D700115
:203F00008D9DF00C9C9DF00C112487010C5E174FC80167E470E00E94D63A9C01009711F16D
:203F20009093270B8093260B2F5F3F4F201B310B2E0D3F1DC9018C5E974F60E070E00E94F2
:203F40001A380E94E4356230710560F48091C20B882341F487EC9BE00E942B2F67E071E0B8
:203F60000E94743380911E0B90911F0B019668E070E00E94B03790931F0B80931E0B809121
:203F8000200B9091210B01969093210B8093200B1092250B1092240B1092230B24C04B33B0
:203FA00011F4B092250B8091250B8823E1F480911E0B90911F0B8C9DF0018D9DF00D9C9DCA
:203FC000F00D1124E20FF31FEC5EF74F40832F5F3F4F3093240B2093230B05C0A0E6CA2E27
:203FE000D12CBB24B39487EC9BE00E942B2F0E946E32882309F4D2C18091200B9091210BAE
:2040000008970CF0CBC187EC9BE00E942B2F0E948232482F8093220B8A3009F066CE71CE5C
:204020008091230B9091240B892B09F0CAC0A5C08CE99BE0B70141E050E00E94B527019746
:2040400019F08FEF9FEF02C0898190E09093C40B8093C30B482F8093220B8A3079F08D30A5
:2040600069F08A3359F02091230B3091240B2F35310524F48F5F9F4F09F060C02091A50B0A
:204080003091A60B4091A70B5091A80B2093BC0B3093BD0B4093BE0B5093BF0B8091B80B75
:2040A0009091B90BA091BA0BB091BB0B281739074A075B0750F01092C00B87EC9BE00E94AF
:2040C0002B2F66E473E00E9474338091230B9091240B009709F475C020911E0B30911F0B83
:2040E000209FF001219FF00D309FF00D1124E80FF91FEC5EF74F10828091250B8823B9F488
:20410000F901EC5EF44FD0828091200B9091210B01969093210B8093200BC901019668E070
:2041200070E00E94B03790931F0B80931E0B1092250B1092240B1092230B27C08B3311F400
:20414000D092250B8091250B8823F9F480911E0B90911F0B809FF001819FF00D909FF00D16
:204160001124E20FF31FEC5EF74F40832F5F3F4F3093240B2093230B08C07E010894E11CE5
:20418000F11C00E610E0DD24D3942091B80B3091B90B4091BA0B5091BB0B8091BC0B9091A5
:2041A000BD0BA091BE0BB091BF0B82179307A407B50738F48091200B9091210B08970CF444
:2041C00037CF8091200B9091210B892B09F491C08091C20B882309F474C020911C0B3091FB
:2041E0001D0B80E690E0289F5001299FB00C389FB00C1124F4E1CF2EF8E0DF2ECA0CDB1CD9
:20420000C60169E573E00E94E13A009709F046C0D6010D900020E9F77D010894E108F10873
:20422000EC18FD0810929E0BC6016EE470E00E94D63A8C01009731F4F501EE0DFF1DED5E6E
:20424000F74F0FC060E270E00E94D63A6C010894C11CD11CC8016AE270E00E94D63AFC011E
:2042600031978DE081838AE0828313828CE99BE0B6010E94A42D80919E0B882341F087ECDE
:204280009BE00E942B2F6DE573E00E94743387EC9BE00E942B2F67E071E010C08CE99BE077
:2042A0000E9496268CE99BE00E94DE261092C20B87EC9BE00E942B2F63E773E00E947433CB
:2042C00002C00E949B148091200B9091210B01979093210B8093200B80911C0B90911D0B9C
:2042E000019668E070E00E94B03790931D0B80931C0B0E94F4060E948B30E0904E0BF0903F
:204300004F0B0091500B1091510B20914A0B30914B0B40914C0B50914D0B621B730B840B52
:20432000950BE616F7060807190798F4E114F1040105110571F01092290B1092280B5D9822
:2043400010922D0B10922C0B5A985E9A5E9A159A5E9A0E948B30E090520BF090530B009188
:20436000540B1091550B20914A0B30914B0B40914C0B50914D0B621B730B840B950BE61639
:20438000F7060807190780F4E114F1040105110559F05E9A5E9A159A5E9A06C08091C00BF5
:2043A000882309F40ECF3CCE0F90CF91DF911F910F91FF90EF90DF90CF90BF90AF900895A8
:2043C000CF92DF92EF92FF920F931F93CF93DF938EED9CE040E052EC61E070E00E947531A3
:2043E0008EED9CE065E873E00E947433E4E1FBE011928BE0EC31F807D9F70C9A149A3D9A18
:204400003F9A229A209A569A5E9A569A5E9A0D9A159A569A5E9A3A98429A3B98439A3C980D
:20442000449A549A5C9A559A529A579A3E9A239A219AC0E0D0E0FE01EF54FC4FE080F180F0
:204440000281138199E6C92E97E0D92ECC0EDD1EFE01E352FC4FC801B70120813181428166
:2044600053810E94CB369B01AC0160E27CEB8EEB9CE40E947C350E94E935F60160837183F9
:204480008283938389E7C82E87E0D82ECC0EDD1EFE01E351FC4F60817181828193810E944F
:2044A0001736A80197010E94CB360E94E935F6016083718382839383B9E8CB2EB7E0DB2EE8
:2044C000CC0EDD1EFE01E350FC4F60817181828193810E941736A80197010E94CB360E942B
:2044E000E935F60160837183828393832496C031D10509F0A0CF0E945414DF91CF911F9142
:204500000F91FF90EF90DF90CF900895FC01673020F086E1858380E00895262F30E060FDB0
:2045200002C0663019F48DB58E7F02C08DB581608DBD8CB58C7F8CBD4CB522FD02C090E0B1
:2045400001C092E036952795822F8170842B892B8CBD81E00895FF920F931F93CF93DF939C
:204560008B010E948B30EB01FF24FA94FEBC0DB407FEFDCF8EB58F3F11F481E008C00E9488
:204580008B306C1B7D0B6017710780F380E0DF91CF911F910F91FF900895FC01848160E001
:2045A0000E94D02F0895FC01848161E00E94D02F0895DC016EBDFA0120E030E00DB407FE63
:2045C000FDCF80818EBD0DB407FEFDCF81818EBD2E5F3F4F329682E02030380779F70DB4DF
:2045E00007FEFDCF8FEF8EBD0DB407FEFDCF8FEF8EBD0DB407FEFDCF8FEF8EBD0DB407FEA5
:20460000FDCF8EB51A968C931A978F71853011F481E0089581E115968C931597CD010E940B
:20462000D32280E00895FF920F931F93CF93DF93EC010E948B308B01FF24FA9409C00E94DD
:204640008B30601B710B6D52714010F08FE00DC0FEBC0DB407FEFDCF8EB58A878F3F79F322
:204660008E3F11F481E006C08DE08D83CE010E94D32280E0DF91CF911F910F91FF900895B2
:20468000CF93DF93EC018E818823D1F08FEF8EBD2F8138854FEF04C00DB407FEFDCF4EBD09
:2046A0002F5F3F4FC901019781509240A8F338872F830DB407FEFDCFCE010E94D3221E8235
:2046C000DF91CF910895DF92EF92FF920F931F93CF93DF93EC01D62E79018A010E944023C7
:2046E000CE010E94CD22CE016CE271E00E94AB228D2D80648EBD0DB407FEFDCF28E130E0E9
:20470000D801C701022E04C0B695A795979587950A94D2F78EBD0DB407FEFDCF2850304009
:204720008FEF283F380761F7DD2011F485E906C088E0D81611F487E801C08FEF8EBD0DB4B2
:2047400007FEFDCF90E02FEF2EBD0DB407FEFDCF8EB587FF02C09150B9F78A87DF91CF9180
:204760001F910F91FF90EF90DF900895CF92DF92EF92FF920F931F93CF93DF93EC017A015B
:204780008B016901411551056105710511F482E137C08B85833039F029E0EE0CFF1C001F13
:2047A000111F2A95D1F7CE0168E1A80197010E946323882311F084E023C0CE016EEFA601FB
:2047C0000E94D9228823E9F0CE0168E572E00E94AB22882311F485E113C0CE016DE020E0D6
:2047E00030E040E050E00E946323882341F48FEF8EBD0DB407FEFDCF8EB5882379F084E13A
:204800008D83CE010E94D32280E0DF91CF911F910F91FF90EF90DF90CF900895CE010E94B8
:20482000D32281E0F2CF8F929F92AF92BF92CF92DF92EF92FF920F931F93CF93DF93EC0184
:204840005A016B0149010115110509F47BC0C801820F931F8150924008F06FC08E81882353
:2048600071F088819981AA81BB81481759076A077B0729F48F8198858816990618F5A882DD
:20488000B982CA82DB828B85833039F069E0AA0CBB1CCC1CDD1C6A95D1F7CE0161E1A60112
:2048A00095010E946323882319F083E08D8345C0CE010E941323882309F43FC018861F8281
:2048C00081E08E838FEF8EBD8F8198852FEF05C00DB407FEFDCF2EBD019688159905C0F38B
:2048E00098878F83D801119720E030E09FEF0BC00DB407FEFDCF8EB5F701E20FF31F8083CA
:204900009EBD2F5F3F4F2A173B0790F30DB407FEFDCF8EB5AE0DBF1D8C932F813885200FF3
:20492000311F38872F838985882319F02050324048F0CE010E94402305C0CE010E94D322DB
:2049400080E001C081E0DF91CF911F910F91FF90EF90DF90CF90BF90AF909F908F90089560
:20496000EF92FF920F931F93790120E030E000E012E00E9413241F910F91FF90EF900895A1
:20498000BF92CF92DF92EF92FF920F931F93CF93DF93EC01B62E1B8619861E821D824C839B
:2049A0000E948B306B018C8161E00E94B22FCE010E94D32286E060E00E94B22F85E061E028
:2049C0000E94B22F87E061E00E94B22F84E061E00E94B22F83E58CBD8DB58E7F8DBD80E057
:2049E0009FEF9EBD0DB407FEFDCF8F5F8A30C9F7CE010E94CD2209C00E948B306C197D0943
:204A0000615D774010F081E05EC0CE0160E020E030E040E050E00E946323182F8A87813002
:204A200059F7CE0168E02AEA31E040E050E00E94632382FF02C01B8711C080E02FEF2EBD53
:204A40000DB407FEFDCF9EB58F5F8430C1F79A879A3A11F082E037C082E08B878B85823092
:204A600021F0EE24FF2487010FC0E12CF12C012D70E4172F09C00E948B306C197D09615DB8
:204A8000774010F088E01FC0CE0167E320E030E040E050E00E946323CE0169E2A80197011C
:204AA0000E9463238A87882331F78B85823031F5CE016AE320E030E040E050E00E9463235E
:204AC000882339F086E08D83CE010E94D32280E01CC08FEF8EBD0DB407FEFDCF8EB5807C50
:204AE000803C11F483E08B8780E09FEF9EBD0DB407FEFDCF2EB58F5F8330C1F7CE010E94F8
:204B0000D322CE016B2D0E948622DF91CF911F910F91FF90EF90DF90CF90BF900895CF93A5
:204B2000DF93EC01DB0180E090E020E2FD01E80FF91F208301968B309105C1F757E040E0C1
:204B400021C02E3219F08CE790E007C05A3019F15AE048E017C03217F1F0FC010196349111
:204B60003323C9F75417B8F02132A8F02F3798F4822F81568A3108F42052FD01E40FF11D7F
:204B800020834F5F29912223E1F690E08C91803219F091E001C090E0892FDF91CF910895DF
:204BA0006F927F928F929F92AF92BF92CF92DF92EF92FF920F931F93CF93DF93EC017A018B
:204BC0008B012C81222309F480C08A899B89AC89BD8984179507A607B70708F476C085C04F
:204BE000E114F1040105110549F41D821E821F82188619861A861B861C8665C029853A85E0
:204C00004B855C85EA8DFB8D858590E00996215030404040504039014A01082E04C0969431
:204C20008794779467940A94D2F72F5F3F4F4F4F5F4F0894E108F108010911095701680121
:204C400004C0D694C794B794A7948A95D2F70894E11CF11C011D111DA614B704C804D9044D
:204C600028F0211531054105510549F48E899F89A88DB98D8D839E83AF83B88716C0A618E7
:204C8000B708C808D90811C04D815E816F8178858A8D9B8D94010E9443030894A108B1087F
:204CA000C108D108882331F410C085E0882E912C8C0E9D1EA114B104C104D10429F7E986F2
:204CC000FA860B871C8781E001C080E0DF91CF911F910F91FF90EF90DF90CF90BF90AF9013
:204CE0009F908F907F906F900895223009F078CFE6CFCF93DF93EC01462F6D857E858F8535
:204D000098890E942701882319F420E030E00AC08989282F30E095E0220F331F9A95E1F79E
:204D2000245D3A4FC901DF91CF9108950F931F93CF93DF938C01FC0184818823C9F1838112
:204D400087FF33C0C80161E00E947926EC01009779F1F8018481823040F482899389A48969
:204D6000B5898C8F9D8FAE8FBF8FF80186899789A08DB18D9B8F8A8FCD01AA27BB279D8BA4
:204D80008C8BE091C50BF091C60B309751F0BE016A5E7F4FCE0148960995888D998D9B8B60
:204DA0008A8BF80183818F7783830E94C80001C080E0DF91CF911F910F910895CF93DF93B9
:204DC000EC010E949626882311F01C8281E0DF91CF9108956F927F928F929F92AF92BF927A
:204DE000CF92DF92EF92FF920F931F93DF93CF9300D000D0CDB7DEB77C015A016B01DC01CD
:204E000014968C911497813009F08FC013968C9181FF8BC09EC00097A105B10511F481E0DF
:204E200085C0F7016184728483849484C701B601A5010E94D025882309F477C0D7015A96D8
:204E40008D919C915B97A114B104C104D10489F456964D915D916D917C9159970E94B60386
:204E6000882309F462C0F701168A178A108E118E3DC0D70115964D915D916D917C911897EC
:204E80009E012F5F3F4F0E944303882309F44DC0D7015A96ED91FC915B9749815A816B8164
:204EA0007C818789803129F088EF9FEFAFEFBFE004C088EF9FEFA0E0B0E0481759076A07D0
:204EC0007B07A0F4CF010E94B603882371F1F7014581568167817085828D938D0FEF1FEFD7
:204EE0002FEF3FE00E94A7028823F9F0D7015296AD92BD92CD92DC92559713968C9113971F
:204F0000806813968C93C7010E949626882369F0B601A5016A147B048C049D0410F4B40173
:204F2000A301C7010E94D02501C080E00F900F900F900F90CF91DF911F910F91FF90EF90A3
:204F4000DF90CF90BF90AF909F908F907F906F900895F70182899389A489B589841795073B
:204F6000A607B70708F057CFE0CF2F923F924F925F926F927F928F929F92AF92BF92CF923E
:204F8000DF92EF92FF920F931F93CF93DF93EC012A018C81882309F4C6C08B8180FFC3C005
:204FA000D8C025014E185F084B0175E0272E312C2C0E3D1E3201B1C029853A854B855C85BC
:204FC0006FEFA62E61E0B62EA222B3228C8179018A0199E016950795F794E7949A95D1F712
:204FE000EA8DFB8D823049F4428D538D648D758D4E0D5F1D601F711F3FC0D480DA94DE207C
:20500000A114B104D9F4DD20C9F4211531054105510549F48E899F89A88DB98D8D839E836F
:20502000AF83B8870BC04D815E816F817885CF0191010E944303882309F475C0EA8DFB8D74
:205040004D815E816F8178854250504060407040058404C0440F551F661F771F0A94D2F7AE
:2050600086859785A089B189480F591F6A1F7B1F4D0D511D611D711D80E092E08A199B09C7
:2050800063018615970508F46C018B8186FD06C080E0C81682E0D80609F073C08091AD034C
:2050A0009091AE03A091AF03B091B003481759076A077B0709F465C080912C0790912D07DA
:2050C0009501860174010E941324882361F18C0C9D1C12C09501245D3A4FA9014C0D5D1D28
:2050E000D401F90102C081918D93E417F507D9F7E21BF30B8E0E9F1E960140E050E08985DD
:205100009A85AB85BC85820F931FA41FB51F89879A87AB87BC876C187D086114710409F093
:205120004BCFA20102C04FEF5FEFCA01DF91CF911F910F91FF90EF90DF90CF90BF90AF900F
:205140009F908F907F906F905F904F903F902F900895AA88BB88CC88DD88E984FA840B8551
:205160001C859A0140E050E0D601C5018E199F09A00BB10B82179307A407B50708F411CFDA
:2051800013CFCB01BA0140E00E942701882309F0A1CFC9CFCF92DF92EF92FF920F931F93D8
:2051A000DF93CF930F92CDB7DEB76C01FC018481823070F0E184F28403851485C601BE015E
:2051C0006F5F7F4F41E050E00E94B527019769F020E030E0C9010F90CF91DF911F910F91DA
:2051E000FF90EF90DF90CF900895F60181859285A385B4854F96A11DB11D81879287A38705
:20520000B487F5E016950795F794E794FA95D1F78E2D8F70282F30E0E5E0220F331FEA95F2
:20522000E1F7245D3A4FD6CFDF93CF9300D00F92CDB7DEB7282F6AE00E94A437805D898382
:20524000822F0E94A437905D9A831B8287EC9BE00E942B2FBE016F5F7F4F0E9445330F907B
:205260000F900F90CF91DF910895EF92FF920F931F938C01812F8695869586950E941429B0
:20528000B7ECEB2EBBE0FB2EC7010E942B2F6AE30E943D33C801A5E096958795AA95E1F7BF
:2052A0008F730E941429C7010E942B2F6AE30E943D330F711070802F880F0E9414291F9115
:2052C0000F91FF90EF900895EF92FF920F931F937C0107EC1BE0C8010E942B2FB701672F9F
:2052E000772766956454784F0E942634C8010E942B2F6DE20E943D33C70125E09695879560
:205300002A95E1F78F700E941429C8010E942B2F6DE20E943D338E2D8F710E9414291F91A8
:205320000F91FF90EF900895DF92EF92FF920F931F93CF93DF937C01D62EEC0110E000E039
:205340008881803291F0083041F487EC9BE00E942B2F6EE20E943D331F5F87EC9BE00E944A
:205360002B2F68810E9435331F5F0F5F21960B3039F7F70183858871803171F487EC9BE0D5
:205380000E942B2F6FE205C087EC9BE00E942B2F60E20E943D331F5F1D15B0F3DF91CF919A
:2053A0001F910F91FF90EF90DF9008950F931F93CF93DF93EC018B018C81882309F041C030
:2053C000FB0187898031B1F482E08C831E8A1F8A188E198E808D918DA0E0B0E045E0880F65
:2053E000991FAA1FBB1F4A95D1F78A8B9B8BAC8BBD8B15C0803229F583E08C83FB01428D0F
:20540000538D648D758D4E8B5F8B688F798F9E012E5E3F4FC8010E940F04882391F01B8FEA
:205420000A8F81E08B831D821E821F82188619861A861B861C861D861E861F86188A198A33
:2054400001C080E0DF91CF911F910F9108951F93CF93DF93EC01142FE62FF0E075E0EE0F81
:20546000FF1F7A95E1F7E45DFA4F8385817121F0842F827409F054C0698B8091AD03909106
:20548000AE03A091AF03B091B0038D879E87AF87B88B84899589A0E0B0E0BC0155274427F3
:2054A000828D938DA0E0B0E0482B592B6A2B7B2B4E8B5F8B688F798F838590E08871907048
:2054C000009751F4848D958DA68DB78D8A8B9B8BAC8BBD8B81E00CC0409711F59E012E5E57
:2054E0003F4F8A8D9B8D0E940F048823C9F084E08C83812F8F708B831D821E821F82188618
:2055000019861A861B861C8616FD02C081E009C0CE0140E050E060E070E00E94EA2601C0E8
:2055200080E0DF91CF911F910895DF92EF92FF920F931F93CF93DF938C01EB017A01D22E4F
:20554000FC018481882341F5822F8073803321F18A8D9B8D938F828FE5E0440F551FEA9582
:20556000E1F760E070E0CE010E94D0258823A1F0CE010E94CA28FC01009771F0808188231D
:2055800059F0853E49F08E3239F06E2D6F70C8014D2D0E94272A01C080E0DF91CF911F918C
:2055A0000F91FF90EF90DF9008952F923F924F925F926F927F928F929F92AF92BF92CF9276
:2055C000DF92EF92FF920F931F93DF93CF93CDB7DEB76E970FB6F894DEBF0FBECDBF6C014E
:2055E0006D8FE42EFC0115821682178210861186128613861486862F90E063E0462E512C87
:205600004822592251E0652E712C6822792244E0842E912C882299221E010894211C311CE2
:205620002E2D2E5F2E8F32E0A32EB12CA822B9228BC0F8018081882309F48DC0853E09F466
:2056400083C08E3209F480C0838583FD7DC0FF2408C087EC9BE00E942B2F60E20E943D331C
:20566000F394FE14B1F74114510411F460E001C06EE0C8010E9494296114710489F0F80167
:20568000808D918D0E94642987EC9BE00E942B2F60E20E943D33F801868997890E9435294A
:2056A000F801838588718031A9F0A114B10491F087EC9BE00E942B2F60E20E943D3387EC0A
:2056C0009BE00E942B2FF801448D558D668D778D0E94173487EC9BE00E942B2F0E945D33A7
:2056E0008114910489F1F80183858871803161F5F60181859285A385B48525E0B695A79504
:20570000979587952A95D1F78C0184E295E09A8389831D82A80141505040C101B60121E046
:205720000E94952A882329F0C1016D8D4E8D0E94D52A85E0000F111F8A95E1F7A80160E088
:2057400070E0C6010E94D025C6010E94CA288C01009709F06ECF6E960FB6F894DEBF0FBE27
:20576000CDBFCF91DF911F910F91FF90EF90DF90CF90BF90AF909F908F907F906F905F90C8
:205780004F903F902F900895CF93DF93EC019C012B5F3F4F8A8D9B8D41E050E060E070E069
:2057A0000E947E048823A1F08E899F89A88DB98D0097A105B10559F48D819E81AF81B885F5
:2057C0008E8B9F8BA88FB98F8B8180688B8381E0DF91CF9108952F923F924F925F927F92C2
:2057E0008F929F92AF92BF92CF92DF92EF92FF920F931F93DF93CF9300D000D000D0CDB7C5
:20580000DEB76C01162F072F5E834D83DC0114968C911497813009F075C113968C9181FFE5
:2058200071C18FC1F601428953896489758981859285A385B48584179507A607B70731F01C
:20584000C6010E94D025882309F45CC1812F902F9C0129012D803E8019C1D6015A96ED9165
:20586000FC915B97DA01C90119E0B695A795979587951A95D1F774807A9478227FEF872E06
:2058800071E0972E82229322772009F050C08114910409F04CC0D60115964D915D916D917E
:2058A0007C911897411551056105710581F456968D919D910D90BC91A02D0097A105B1054D
:2058C00059F1F60185839683A783B08730C0CF019E012F5F3F4F0E944303882319F440E0CA
:2058E00050E016C129813A814B815C81D6015A96ED91FC915B978789803129F088EF9FEFF0
:20590000AFEFBFE004C088EF9FEFA0E0B0E0281739074A075B0730F0C6010E94C42B88231C
:2059200031F4F0C0F601258336834783508780E092E08819990951018215930508F45C01AA
:20594000D6015A96ED91FC915B971596ED90FD900D911C9118978EEF9FEFAFEFBFEFE80E87
:20596000F91E0A1F1B1F058404C0EE0CFF1C001F111F0A94D2F786859785A089B189E80E15
:20598000F91E0A1F1B1FE70CF11C011D111D90E0A91692E0B90651F58091AD039091AE0308
:2059A000A091AF03B091B0038E159F05A007B10761F48FEF9FEFAFEFBFEF8093AD039093D7
:2059C000AE03A093AF03B093B00380912C0790912D07B801A70192010E94B623882309F48B
:2059E00091C0A0E0B2E04A0E5B1E3EC08114910409F5F60121853285438554858289938931
:205A0000A489B589281739074A075B0798F00E94C800882309F476C0E092AD03F092AE03C4
:205A20000093AF031093B00380912E07816080932E0708C0C801B70141E00E94270188237D
:205A400009F460C09401245D3A4FA9014A0D5B1DD201F90102C08D918193E417F507D9F789
:205A6000E21BF30B4E0E5F1E2A183B08950140E050E0F60181859285A385B485820F931F2F
:205A8000A41FB51F81879287A387B487D60119962D913D914D915C911C972114310409F0F6
:205AA000DCCE52968D919D910D90BC91A02D82179307A407B50748F4F601228B338B448B4A
:205AC000558B83818068838311C08091C50B9091C60B892B59F08D819E81892B39F0D60172
:205AE00013968C911397806813968C93F601838183FF05C0C6010E949626882319F04D819D
:205B00005E8106C081E0D60112968C934FEF5FEFCA0126960FB6F894DEBF0FBECDBFCF9127
:205B2000DF911F910F91FF90EF90DF90CF90BF90AF909F908F907F905F904F903F902F9082
:205B4000089582FD6FCE82CEDB010D900020E9F71197A61BB70BAD010E94EB2B0895DF9383
:205B6000CF930F92CDB7DEB76983BE016F5F7F4F41E050E00E94EB2B0F90CF91DF910895AD
:205B8000DF92EF92FF920F931F93CF93DF93EC010E94C42B882309F44EC0EA8DFB8DED80BA
:205BA000FE800F8118858EEF9FEFAFEFBFEFE80EF91E0A1F1B1F058404C0EE0CFF1C001FF2
:205BC000111F0A94D2F786859785A089B189E80EF91E0A1F1B1FD4800894E108F108010958
:205BE00011090BC0C801B7016D0D711D811D911D0E9403018823F9F0DA94DD2099F7EA8D3F
:205C0000FB8D20E032E040E050E0058404C0220F331F441F551F0A94D2F78A899B89AC8920
:205C2000BD89820F931FA41FB51F8A8B9B8BAC8BBD8B81E001C080E0DF91CF911F910F91E8
:205C4000FF90EF90DF9008956F927F928F929F92AF92BF92CF92DF92EF92FF920F931F93FC
:205C6000DF93CF93CDB7DEB72B970FB6F894DEBF0FBECDBF5C016B01822EDC0114968C9111
:205C8000882309F0D2C0CA018E010F5F1F4FB8010E948F25882309F4C8C0F601828D938D33
:205CA000D5015B969C938E935A971582168217821086D60119961D921D921D921C921C978A
:205CC0009924380141C0C6010E94CA28FC01009709F4ABC085E016950795F794E7948A95A5
:205CE000D1F71E2D1F708081882311F0853ED1F4992091F4D50151961C9351972091AD03DA
:205D00003091AE034091AF035091B0031D962D933D934D935C9350978081882399F499240B
:205D2000939421C0C301BF014BE050E00E94C93A009751F4882D8073803309F476C0C501A7
:205D4000612F6FC099249394F601E184F2840385148582899389A489B589E816F9060A070D
:205D60001B0708F4B0CF882D8271823109F05DC0992041F0C50161E00E9479268C010097BF
:205D800089F453C0D60114968C91823009F44DC0C6010E94C02D882309F447C0F501118A83
:205DA0000CE215E080E2D8011D928A95E9F7D801FE0131968BE001900D928150E1F7E091C3
:205DC000C50BF091C60B309739F0B801625F7F4FC8014096099509C081E298E2F801918B71
:205DE000808B80E098E097878687D80150968D919C91519753969C938E93529759969C9363
:205E00008E9358971E968D919C911F9757969C938E9356970E94C800882339F0C501F50199
:205E20006189482D0E94272A01C080E02B960FB6F894DEBF0FBECDBFCF91DF911F910F91C7
:205E4000FF90EF90DF90CF90BF90AF909F908F907F906F900895FC018081918108958EEDB7
:205E60009CE09093C80B8093C70B0895CB01642F0E94033B0895CB010E94FB3A08959091F1
:205E8000CF049295990F990F907C8770892B80937C0080917A00806480937A0080917A00EB
:205EA00086FDFCCF2091780040917900942F80E030E0282B392BC90108951F93CF93DF934A
:205EC000182FEB0161E00E94B22FE12FF0E0E552FF4F8491833051F48091800080688093CD
:205EE0008000D0938900C093880038C0843051F480918000806280938000D0938B00C09323
:205F00008A002CC0813029F484B5806884BDC7BD25C0823029F484B5806284BDC8BD1EC0E4
:205F2000863041F48091B00080688093B000C093B30014C0873041F48091B000806280938E
:205F4000B000C093B4000AC0C038D1051CF4812F60E002C0812F61E00E94D02FDF91CF91CE
:205F60001F910895282F30E0C90185549F4FFC01949125563F4FF9018491882381F0E82F6F
:205F8000F0E0E457FF4FE491F0E0662329F4808190958923808308958081892B80830895F6
:205FA000482F50E0CA0185529F4FFC012491CA0185549F4FFC01949145565F4FFA0134913B
:205FC0003323C1F1222331F1213019F484B58F7704C0223021F484B58F7D84BD1BC02330D6
:205FE00021F4809180008F7705C0243031F4809180008F7D809380000DC0263021F480913E
:20600000B0008F7705C0273029F48091B0008F7D8093B000E32FF0E0EF56FF4FE491F0E047
:20602000662329F4808190958923808308958081892B808308951F920F920FB60F92112406
:206040002F938F939F93AF93BF938091CA0B9091CB0BA091CC0BB091CD0B0196A11DB11D75
:206060008093CA0B9093CB0BA093CC0BB093CD0B8091CE0B9091CF0BA091D00BB091D10B0C
:206080008050904CAF4FBF4F8093CE0B9093CF0BA093D00BB093D10B27C08091CE0B909140
:2060A000CF0BA091D00BB091D10B80589E43A040B0408093CE0B9093CF0BA093D00BB0931A
:2060C000D10B8091D20B9091D30BA091D40BB091D50B0196A11DB11D8093D20B9093D30BB2
:2060E000A093D40BB093D50B8091CE0B9091CF0BA091D00BB091D10B81589E43A040B040D3
:2061000060F6BF91AF919F918F912F910F900FBE0F901F9018958FB7F8942091D20B309101
:20612000D30B4091D40B5091D50B8FBFB901CA0108956FB7F89486B590E0A0E0B0E0A89BF0
:2061400008C00097A105B10521F480E091E0A0E0B0E02091CA0B3091CB0B4091CC0B5091E8
:20616000CD0B6FBF542F432F322F2227280F391F4A1F5B1F82E0220F331F441F551F8A952D
:20618000D1F7B901CA010895789484B5826084BD84B5816084BD85B5826085BD85B58160D9
:2061A00085BDEEE6F0E0808181608083E1E8F0E0808182608083808181608083E0E8F0E018
:2061C000808181608083E1EBF0E0808184608083E0EBF0E0808181608083EAE7F0E0808134
:2061E000846080838081826080838081816080838081806880831092C10008950F931F93AD
:20620000CF93DF93482FFB018B0100581F4FD801CD91DC91CE01019660E870E00E94B037BA
:206220009C01EE57FF4F80819181E258F0402817390731F0CE0FDF1F4883F801318320831B
:20624000DF91CF911F910F9108951F920F920FB60F9211242F933F934F935F936F937F9318
:206260008F939F93AF93BF93EF93FF938091C60066ED7BE00E94FE30FF91EF91BF91AF912D
:206280009F918F917F916F915F914F913F912F910F900FBE0F901F9018951F920F920FB6C0
:2062A0000F9211242F933F934F935F936F937F938F939F93AF93BF93EF93FF938091CE00B1
:2062C0006AE57CE00E94FE30FF91EF91BF91AF919F918F917F916F915F914F913F912F91E3
:2062E0000F900FBE0F901F9018955F926F927F928F929F92AF92BF92CF92DF92EF92FF926C
:206300000F931F93CF93DF93EC013A014B01413482E458078FE0680780E078070CF07FC0AF
:2063200060E874E88EE190E0A40193010E94E5372150304040405040CA01B90122E030E05B
:2063400040E050E00E94E53759016A01A6019501209530954095509594E0220F331F441F9F
:20636000551F9A95D1F760E074E284EF90E00E94E537CA01B9012FEF30E040E050E00E94D6
:206380008537A40193010E94E537C90181509F4F181619061CF4522E5A9403C055245394D3
:2063A000521A60E079E08DE390E0A40193010E94E5372150304040405040CA01B90122E089
:2063C00030E040E050E00E94E537209530954095509583E0220F331F441F551F8A95D1F7C7
:2063E00060E074E284EF90E00E94E537CA01B9012FEF30E040E050E00E948537A4019301CC
:206400000E94E537C90181509F4F181619061CF4822F815002C081E0821B851500F5E8859A
:20642000F98581E090E00A8802C0880F991F0A94E2F7808360E079E08DE390E0A40193013E
:206440000E94E5372150304040405040CA01B90122E030E040E050E00E94E53704C0E885B7
:20646000F98510829501EC81FD813083EE81FF812083EA85FB85208141E050E0CA010E8408
:2064800002C0880F991F0A94E2F7282B2083EA85FB852081CA010F8402C0880F991F0A94E1
:2064A000E2F7282B2083EA85FB858081088802C0440F551F0A94E2F7842B8083DF91CF910B
:2064C0001F910F91FF90EF90DF90CF90BF90AF909F908F907F906F905F900895DC01129695
:2064E000ED91FC911397E058FF4F8191919180589F4F20813181821B930B60E870E00E949F
:20650000B0370895CF93DF93DC011296ED91FC911397EF01CE57DF4F48815981E058FF4F7D
:2065200080819181E058F0408417950719F42FEF3FEF0CC0E40FF51F2081CA01019660E832
:2065400070E00E94B0379983888330E0C901DF91CF910895DC011296ED91FC911397EE5775
:20656000FF4F80819181929382930895FC01A085B18521898C9190E0022E02C0959587951C
:206580000A94E2F780FFF6CF0484F585E02D608308952AE235E03093DF0C2093DE0C86EDD2
:2065A0009BE09093E10C8093E00C85EC90E09093E30C8093E20C84EC90E09093E50C809356
:2065C000E40C80EC90E09093E70C8093E60C81EC90E09093E90C8093E80C86EC90E09093D3
:2065E000EB0C8093EA0CE4E0E093EC0C73E07093ED0C67E06093EE0C55E05093EF0C41E0B5
:206600004093F00C3093F20C2093F10C8AE59CE09093F40C8093F30C8DEC90E09093F60C0C
:206620008093F50C8CEC90E09093F80C8093F70C88EC90E09093FA0C8093F90C89EC90E017
:206640009093FC0C8093FB0C8EEC90E09093FE0C8093FD0CE093FF0C7093000D6093010D33
:206660005093020D4093030D0895DC01ED91FC910190F081E02D09950895DC01ED91FC918E
:206680000190F081E02D099508950F931F93CF93DF938C01EB0109C02196D801ED91FC91AB
:2066A0000190F081E02DC801099568816623A1F7DF91CF911F910F9108950F931F938C01BC
:2066C000DC01ED91FC910190F081E02D6DE00995D801ED91FC910190F081E02DC8016AE0D2
:2066E00009951F910F9108950F931F938C010E944533C8010E945D331F910F9108952F926B
:206700003F924F925F926F927F928F929F92AF92BF92CF92DF92EF92FF920F931F93DF9336
:20672000CF93CDB7DEB7A0970FB6F894DEBF0FBECDBF1C016A017B014115510561057105D4
:2067400049F4DC01ED91FC910190F081E02D60E3099554C0882499245401422E55246624DF
:20676000772401E010E00C0F1D1F080D191DC701B601A30192010E94C337F8016083089441
:20678000811C911CA11CB11CC701B601A30192010E94C337C901DA016C017D01C114D10499
:2067A000E104F104F1F681E0E82EF12CEC0EFD1EE80CF91C3E010894611C711CD501C401E6
:2067C0000197A109B1096C01C818D90814C0F601EE0DFF1D60816A3010F4605D01C0695CEB
:2067E000D101ED91FC910190F081E02DC10109950894E108F1086E147F0449F7A0960FB68F
:20680000F894DEBF0FBECDBFCF91DF911F910F91FF90EF90DF90CF90BF90AF909F908F901E
:206820007F906F905F904F903F902F9008952AE00E947F3308950F931F938C010E94173488
:20684000C8010E945D331F910F910895AB0160E070E00E9417340895EF92FF920F931F9324
:20686000CF93DF93EC017A018B0177FF0FC0E881F9810190F081E02D6DE2099510950095F2
:20688000F094E094E11CF11C011D111DCE01B801A7012AE00E947F33DF91CF911F910F91FC
:2068A000FF90EF9008950F931F938C010E942C34C8010E945D331F910F910895AB01662729
:2068C00057FD6095762F0E942C3408950F931F938C01AB01662757FD6095762F0E942C3421
:2068E000C8010E945D331F910F9108959F92AF92BF92CF92DF92EF92FF920F931F93CF9353
:20690000DF93EC017A018B01922ECB01BA0120E030E040E050E00E947835882364F4E881AF
:20692000F9810190F081E02DCE016DE2099517FB109517F9109520E030E040E05FE3AA2466
:206940000BC0CA01B90120E030E040E251E40E947C359B01AC01A394A91498F3C801B701E4
:206960000E9414355B016C010E94E9357B018C01CE01B801A7010E941734992029F0CE01DC
:206980006BEA73E00E944533C801B7010E9415369B01AC01C601B5010E94133520C020E037
:2069A00030E040E251E40E94CB367B018C010E94E4355B016C01CC24B7FCC094DC2CCE0172
:2069C000B601A5010E942C34C601B5010E9417369B01AC01C801B7010E9413359A94992051
:2069E000F1F6DF91CF911F910F91FF90EF90DF90CF90BF90AF909F90089522E00E9476340C
:206A000008950F931F938C010E94FD34C8010E945D331F910F9108950E94C4300E94E02104
:206A20000E94601EFDCF5058BB27AA270ED075C166D130F06BD120F031F49F3F11F41EF43E
:206A40005BC10EF4E095E7FB51C1E92F77D180F3BA17620773078407950718F071F49EF501
:206A60008FC10EF4E0950B2EBA2FA02D0B01B90190010C01CA01A0011124FF27591B99F038
:206A8000593F50F4503E68F11A16F040A22F232F342F4427585FF3CF469537952795A795CA
:206AA000F0405395C9F77EF41F16BA0B620B730B840BBAF09150A1F0FF0FBB1F661F771FF9
:206AC000881FC2F70EC0BA0F621F731F841F48F4879577956795B795F7959E3F08F0B3CF7A
:206AE0009395880F08F09927EE0F979587950895D9D008F481E008950CD00FC107D140F0E6
:206B0000FED030F021F45F3F19F0F0C0511139C1F3C014D198F39923C9F35523B1F3951B58
:206B2000550BBB27AA2762177307840738F09F5F5F4F220F331F441FAA1FA9F333D00E2E66
:206B40003AF0E0E830D091505040E695001CCAF729D0FE2F27D0660F771F881FBB1F261794
:206B600037074807AB07B0E809F0BB0B802DBF01FF2793585F4F2AF09E3F510568F0B6C038
:206B800000C15F3FECF3983EDCF3869577956795B795F7959F5FC9F7880F911D96958795CD
:206BA00097F90895E1E0660F771F881FBB1F621773078407BA0720F0621B730B840BBA0BBD
:206BC000EE1F88F7E095089504D06894B111D9C00895BCD088F09F5790F0B92F9927B75125
:206BE000A0F0D1F0660F771F881F991F1AF0BA95C9F712C0B13081F0C3D0B1E00895C0C05C
:206C0000672F782F8827B85F39F0B93FCCF3869577956795B395D9F73EF4909580957095E5
:206C200061957F4F8F4F9F4F0895E89409C097FB3EF490958095709561957F4F8F4F9F4F4F
:206C40009923A9F0F92F96E9BB279395F695879577956795B795F111F8CFFAF4BB0F11F4AD
:206C600060FF1BC06F5F7F4F8F4F9F4F16C0882311F096E911C0772321F09EE8872F762F14
:206C800005C0662371F096E8862F70E060E02AF09A95660F771F881FDAF7880F96958795D8
:206CA00097F90895990F0008550FAA0BE0E8FEEF16161706E807F907C0F012161306E40715
:206CC000F50798F0621B730B840B950B39F40A2661F0232B242B252B21F408950A2609F48C
:206CE000A140A6958FEF811D811D089597F99F6780E870E060E008959FEF80EC089500243B
:206D00000A941616170618060906089500240A9412161306140605060895092E0394000C23
:206D200011F4882352F0BB0F40F4BF2B11F460FF04C06F5F7F4F8F4F9F4F089557FD905810
:206D4000440F551F59F05F3F71F04795880F97FB991F61F09F3F79F08795089512161306D5
:206D60001406551FF2CF4695F1DF08C0161617061806991FF1CF8695710561050894089542
:206D8000E894BB2766277727CB0197F908958ADF08F48FEF08950BD0C0CFB1DF28F0B6DF4A
:206DA00018F0952309F0A2CFA7CF1124EACFC6DFA0F3959FD1F3950F50E0551F629FF001DB
:206DC000729FBB27F00DB11D639FAA27F00DB11DAA1F649F6627B00DA11D661F829F222794
:206DE000B00DA11D621F739FB00DA11D621F839FA00D611D221F749F3327A00D611D231F21
:206E0000849F600D211D822F762F6A2F11249F5750408AF0E1F088234AF0EE0FFF1FBB1FD5
:206E2000661F771F881F91505040A9F79E3F510570F05CCFA6CF5F3FECF3983EDCF386950F
:206E400077956795B795F795E7959F5FC1F7FE2B880F911D9695879597F9089511F40EF437
:206E60004BCF3EC073DFD0F39923D9F3CEF39F57550B87FF43D00024A0E640EA9001805870
:206E80005695979528F4805C660F771F881F20F026173707480730F4621B730B840B202960
:206EA00031294A2BA69517940794202531254A2758F7660F771F881F20F02617370748079B
:206EC00030F4620B730B840B200D311D411DA09581F7B901842F9158880F969587950895BD
:206EE0009F3F31F0915020F4879577956795B795880F911D9695879597F908959150504004
:206F0000660F771F881FD2F70895629FD001739FF001829FE00DF11D649FE00DF11D929F39
:206F2000F00D839FF00D749FF00D659FF00D9927729FB00DE11DF91F639FB00DE11DF91FAB
:206F4000BD01CF0111240895991B79E004C0991F961708F0961B881F7A95C9F780950895CA
:206F600097FB092E07260AD077FD04D049D006D000201AF4709561957F4F0895F6F7909564
:206F800081959F4F0895A1E21A2EAA1BBB1BFD010DC0AA1FBB1FEE1FFF1FA217B307E407F3
:206FA000F50720F0A21BB30BE40BF50B661F771F881F991F1A9469F760957095809590959F
:206FC0009B01AC01BD01CF01089597FB092E05260ED057FD04D0D7DF0AD0001C38F4509586
:206FE0004095309521953F4F4F4F5F4F0895F6F790958095709561957F4F8F4F9F4F089571
:20700000AA1BBB1B51E107C0AA1FBB1FA617B70710F0A61BB70B881F991F5A95A9F7809538
:207020009095BC01CD010895EE0FFF1F0590F491E02D0994A0E0B0E0E0E2F8E30C941A3B82
:20704000EC015B016115710519F0FB0191838083F9908F2D90E00E94A93A892BC9F7FDE252
:20706000FF1621F4F990EE24E39405C02BE2F21609F4F990EE248E0101501040C8016BEF0F
:2070800070E043E050E00E94B13A892B01F58E010E5F1F4FC8016EEF70E045E050E00E943F
:2070A000B13A892B19F48E01095F1F4FA114B10419F0F50111830083E0FC04C070E090E0DF
:2070C00080E814C070E090E080E86FEF08C1C80163E071E043E050E00E94B13A892B69F4D7
:2070E000A114B10429F470E090E080EC6FE7F7C02296F501D183C083F6CF8824992440E03D
:2071000050E060E070E0EF2DE053EA30A0F5F2E0EF2A8E2D90E09C0128703070E2FE06C020
:20712000232B79F50894811C911C2BC0232B19F0089481089108DB01CA0112E0880F991FC5
:20714000AA1FBB1F1A95D1F7480F591F6A1F7B1F440F551F661F771F4E0F511D611D711D6A
:20716000483929E9520729E9620729E1720748F084E0E82A06C0EE3F31F4E3FC39C098E00F
:20718000E92AF990C0CFE53311F0E53189F529912D3219F4E0E1EE2A05C02B3219F081E08C
:2071A00090E003C0299182E090E0E22FE053EA3018F0C81BD90B1CC020E030E0FCE02038C3
:2071C0003F075CF4C901880F991F880F991F280F391F220F331F2E0F311DE991E053EA304D
:2071E00068F3E4FE03C0309521953F4F820E931ECE2CDD24E1FE07C0A114B10421F0219771
:20720000F501D183C083CB01BA010E9415367B018C01F3E0CF22DD2423E0C216D10421F4DA
:2072200017FB109517F9109557016801C801B70120E030E040E050E00E947835882309F449
:207240004AC097FE0DC02AE1E22E21E0F22E9094819491089394C0E2D0E000E010E012C099
:2072600092E3E92E91E0F92EF6CFF7012591359145915491C601B5010E94CB365B016C010D
:207280008C1A9D0A8C169D0684F7D595C7950F5F1F4F0630110529F08CEF9FEFE80EF91EC4
:2072A000F1CFC501D6017C018D018C2D880F8D2D881F8F3F51F0C601B50120E030E040E0F9
:2072C00050E00E947835882331F482E290E09093050D8093040D7E2D9F2D802F612F272F26
:2072E000392F482F562FB901CA01CDB7DEB7ECE00C94363B2F923F925F926F927F928F92F9
:207300009F92AF92BF92CF92DF92EF92FF920F931F93CF93DF938C011B01EA01611571051E
:2073200019F0FB0191838083209749F0CE010297839728F020E030E040E050E0F6C0F80198
:20734000A1908F018A2D90E00E94A93A892BB9F7FDE2AF1631F4F801A1908F015524539479
:2073600007C0FBE2AF1619F4F801A1908F015524209719F0C031D105C1F4F0E3AF1679F423
:20738000F8018081883711F0883549F4F801A1800E5F1F4FF2E05F2AC0E1D0E006C020971B
:2073A00021F480E3A816E9F427C0C830D10531F1C930D10524F4C230D10531F50CC0CA3048
:2073C000D10589F0C031D105F9F4C12CD12CE12CB8E0FB2E28C0C12CD12CE12CA0E4FA2E67
:2073E00022C0CAE0D0E0FCECCF2EFCECDF2EFCECEF2EFCE0FF2E17C0C8E0D0E0C12CD12C50
:20740000E12CE0E1FE2E0FC09E01442737FD4095542F60E070E080E090E80E94C337C9013F
:20742000DA016C017D0120E030E040E050E060E03E01882477FC8094982C70EDB72EBA0CA8
:20744000E9E0EB1570F48A2D81548A3118F499ECB92E06C08A2D81568A3150F589EAB82E93
:20746000BA0C8B2D90E08C179D0714F56F3FE1F0C216D306E406F506B0F0CA01B901A401EF
:2074800093010E9485379B01AC012B0D311D411D511D2130F0E03F07F0E04F07F0E85F0794
:2074A00010F461E001C06FEFF801A1908F01C5CF2114310481F0662331F001501040F10102
:2074C0001183008308C051FE1AC002501040F1011183008314C067FF12C050FC05C02FEFBE
:2074E0003FEF4FEF5FE704C020E030E040E050E882E290E09093050D8093040D16C050FE5D
:2075000008C050954095309521953F4F4F4F5F4F0CC057FF0AC082E290E09093050D80938C
:20752000040D2FEF3FEF4FEF5FE7B901CA01DF91CF911F910F91FF90EF90DF90CF90BF909A
:20754000AF909F908F907F906F905F903F902F900895911166C0803219F089508550D0F77E
:207560000895FB01DC014150504088F08D9181341CF08B350CF4805E659161341CF06B3548
:207580000CF4605E861B611171F3990B0895881BFCCFFB01DC0104C08D910190801921F40D
:2075A00041505040C8F7881B990B0895FC018191861721F08823D9F7992708953197CF01DA
:2075C0000895FB0151915523A9F0BF01DC014D9145174111E1F759F4CD010190002049F019
:2075E0004D9140154111C9F3FB014111EFCF81E090E001970895F999FECF92BD81BDF89ABA
:20760000992780B50895262FF999FECF1FBA92BD81BD20BD0FB6F894FA9AF99A0FBE019605
:2076200008959927882708952F923F924F925F926F927F928F929F92AF92BF92CF92DF9275
:20764000EF92FF920F931F93CF93DF93CDB7DEB7CA1BDB0B0FB6F894DEBF0FBECDBF099428
:207660002A88398848885F846E847D848C849B84AA84B984C884DF80EE80FD800C811B8198
:20768000AA81B981CE0FD11D0FB6F894DEBF0FBECDBFED010895F894FFCF45433A002C2080
:2076A000006F6B00526573656E643A00534420696E6974206661696C00766F6C756D652E68
:2076C000696E6974206661696C6564006F70656E526F6F74206661696C656400533A0042C7
:2076E0006567696E2066696C65206C69737400456E642066696C65206C6973740046696C7D
:2077000065206F70656E65643A002053697A653A0046696C652073656C65637465640066EB
:20772000696C652E6F70656E206661696C6564005344207072696E74696E672062797465B4
:2077400020002F004E6F74205344207072696E74696E67006F70656E206661696C65642C04
:207760002046696C653A20002E0057726974696E6720746F2066696C653A20006F6B205492
:207780003A0020423A006F6B206F3A002C20703A002C20693A002C20643A00543A00464984
:2077A000524D574152455F4E414D453A72727020555549443A00583A00593A005A3A00455E
:2077C0003A00785F6D696E3A004C2000482000795F6D696E3A007A5F6D696E3A00004B70DE
:2077E00020004B6920004B6420005049445F4D415820005049445F495F4D415820004E5AF2
:207800004F4E452000556E6B6E6F776E20636F6D6D616E643A004D3131300053657269616A
:207820006C204572726F723A204C696E65204E756D626572206973206E6F74204C61737426
:20784000204C696E65204E756D6265722B312C204C617374204C696E653A004572726F72CF
:207860003A20636865636B73756D206D69736D617463682C204C617374204C696E653A0023
:207880004572726F723A204E6F20436865636B73756D2077697468206C696E65206E756D60
:2078A0006265722C204C617374204C696E653A004572726F723A204E6F204C696E65204E96
:2078C000756D626572207769746820636865636B73756D2C204C617374204C696E653A007C
:2078E000446F6E65207072696E74696E672066696C65004D3239006572726F722077726963
:2079000074696E6720746F2066696C6500446F6E6520736176696E672066696C652E007363
:2079200074617274004F6B005344004572726F72004E6F204572726F7200486F74656E64E8
:2079400000426564002E00FFFFFFFF71DBB64271DBB64200007A45008063440060EA4600F4
:2079600060EA460000FA430060EA460080BB440080BB440000F0420000C8410000C841CD9B
:20798000CC4C3E00002041E8030000E803000032000000FA000000F4010000F40100003212
:2079A000000000F401000030303030303030302D303030302D303030302D303030302D302E
:2079C000303030303030303030303000FF005000000000400AD7233C0000A04105000100E1
:2079E000A10324002B014700F6006A00D9008D00C600B000B800D300AD00F600A300190125
:207A00009A003C0193005F018C0082018600A5018000C8017A00EB0175000E02700031028A
:207A20006B0054026600770261009A025B00BD025600E002510003034C00260346004903F9
:207A40003F006C0338008F033000B2032600D5031700F80300008B038E0391039703A003C9
:207A6000A70358595A4501DC05010100C0023600D8006B00AF00A0009800D50089000A019D
:207A80007D003F01730074016A00A9016300DE015B001302550048024E007D024700B20214
:207AA0004100E7023A001C03320051032A0086031F00BB031100F003000000000000AF2D4D
:207AC00000000000B632FFFFFFFFFFFFFFFFFFFFFFFFFFFFFFFFFFFFFFFFFFFFFFFFFFFFD8
:207AE000FFFFFFFFFFFFFFFFFFFFFFFFFFFFFFFFFFFFFFFFFFFFFFFFFFFFFFFFFFFFFFFFA6
:207B0000FFFFFFFFFFFFFFFFFFFFFFFFFFFFFFFFFFFFFFFFFFFFFFFFFFFFFFFFFFFFFFFF85
:207B2000FFFFFFFFFFFFFFFFFFFFFFFFFFFFFFFFFFFFFFFFFFFFFFFFFFFFFFFFFFFFFFFF65
:207B4000FFFFFFFFFFFFFFFFFFFFFFFFFFFFFFFFFFFFFFFFFFFFFFFFFFFFFFFFFFFFFFFF45
:20F800000C943E7C0C945B7C0C945B7C0C945B7C0C945B7C0C945B7C0C945B7C0C945B7C4D
:20F820000C945B7C0C945B7C0C945B7C0C945B7C0C945B7C0C945B7C0C945B7C0C945B7C10
:20F840000C945B7C0C945B7C0C945B7C0C945B7C0C945B7C0C945B7C0C945B7C0C945B7CF0
:20F860000C945B7C0C945B7C0C945B7C0C945B7C0C945B7C0C945B7C0C945B7C11241FBE35
:20F88000CFEFD0E1DEBFCDBF11E0A0E0B1E0E6E6FFEF02C005900D92A030B107D9F712E0D4
:20F8A000A0E0B1E001C01D92A930B107E1F70E94537D0C94B27F0C94007CCF93DF93CDB7A7
:20F8C000DEB724970FB6F894DEBF0FBECDBF882309F481E020E0482F55274115510509F4EC
:20F8E0003DC0289A19821A821B821C820BC089819A81AB81BC810196A11DB11D89839A8332
:20F90000AB83BC8389819A81AB81BC8180589E43A040B04060F3289819821A821B821C82DE
:20F920000BC089819A81AB81BC810196A11DB11D89839A83AB83BC8389819A81AB81BC8127
:20F9400080509A4FA040B04060F32F5F822F992787FD9095841795070CF4C3CF19821A8223
:20F960001B821C8289819A81AB81BC8180509147A240B040A0F489819A81AB81BC8101968B
:20F98000A11DB11D89839A83AB83BC8389819A81AB81BC8180509147A240B04060F3249630
:20F9A0000FB6F894DEBF0FBECDBFDF91CF910895EF92FF920F931F93EE24FF2487012898B0
:20F9C0008091C00087FD17C00894E11CF11C011D111D81E0E81689E0F8068DE3080780E064
:20F9E000180770F3E0910001F091010109958091C00087FFE9CF289A8091C600992787FD06
:20FA000090951F910F91FF90EF900895982F8091C00085FFFCCF9093C60008950E94D87C63
:20FA2000803271F0809102018F5F80930201853009F00895E0910001F09101010995089520
:20FA400084E10E94067D80E10E94067D0895CF93C82F0E94D87C803241F0809102018F5FC5
:20FA600080930201853081F40AC084E10E94067D8C2F0E94067D80E10E94067D05C0E09156
:20FA80000001F09101010995CF910895282F90E007C08091C0008823E4F78091C6009F5F8D
:20FAA0009217B8F30895CFEFD0E1DEBFCDBF000094B714BE80916000886180936000109231
:20FAC000600091FF74C189E18093C4001092C50088E18093C10086E08093C2005098589A07
:20FAE000209A83E00E945D7C81E00E945D7C0E94D87C8033B9F18133C1F1803409F456C012
:20FB0000813409F45CC0823409F46EC0853409F471C0803539F1813509F4F3C0823511F151
:20FB2000853509F4D3C0863509F4CBC0843609F465C0843709F4EBC0853709F4D2C08637F1
:20FB400009F44AC0809102018F5F80930201853071F6E0910001F091010109950E94D87CE1
:20FB6000803349F60E940E7DC2CF0E94D87CC82F803241F784E10E94067D81E40E94067DEA
:20FB800086E50E94067D82E50E94067D8C2F0E94067D89E40E94067D83E50E94067D80E5E5
:20FBA0000E94067D80E10E94067DA1CF0E94D87C8638C0F20E94D87C0E940E7D98CF0E9498
:20FBC000D87C803809F407C1813809F400C1823809F4F9C0883921F080E00E94277D87CF9F
:20FBE00083E00E94277D83CF84E10E94467D0E940E7D7DCF85E00E94467DF9CF0E94D87C3F
:20FC0000809306020E94D87C80930502809108028E7F809308020E94D87C853409F44BC0BD
:20FC2000E5E0F1E0119281E0E438F807D9F3D0F3C0E0D0E0809105029091060218161906A2
:20FC400078F405E011E00E94D87CF80181938F0121968091050290910602C817D90798F38D
:20FC60000E94D87C803209F06DCF8091080280FFB6C0C0E0D0E0209105023091060212169E
:20FC80001306B8F4E0910301F0910401A5E0B1E0F999FECFF2BDE1BD8D9180BDFA9AF99A60
:20FCA00031962196C217D30798F3F0930401E093030184E175CF80910802816080930802C7
:20FCC000AFCF84E00E94467D80E087CF0E94D87C809303010E94D87C809304010E940E7DDF
:20FCE00006CF0E94D87C803209F02CCF84E10E94067D8EE10E94067D86E90E94067D8AE077
:20FD00004FCF0E940E7D88E080936000FFCF0E94D87C809306020E94D87C809305020E942C
:20FD2000D87C853409F449C0809108028E7F809308028091030190910401880F991F9093BE
:20FD40000401809303010E94D87C803209F0CFCE84E10E94067DC0E0D0E0209105023091F6
:20FD600006021216130608F01DCFE0910301F09104018091080280FF96C0F999FECFF2BD5D
:20FD8000E1BDF89A80B50E94067DE0910301F09104013196F0930401E09303012091050260
:20FDA000309106022196C217D30718F3FBCEE0910001F0910101099586CE80910802816059
:20FDC00080930802C0CF80E10E94277D90CE81E00E94277D8CCE82E00E94277D88CE809162
:20FDE000030190910401880F991F90930401809303018091050280FF09C0809105029091B2
:20FE0000060201969093060280930502F999FECF1127E0910301F0910401C5E0D1E0809105
:20FE2000050290910602103091F40091570001700130D9F303E000935700E8950091570045
:20FE400001700130D9F301E100935700E895099019900091570001700130D9F301E00093DF
:20FE60005700E8951395103898F011270091570001700130D9F305E000935700E8950091CB
:20FE8000570001700130D9F301E100935700E8953296029709F0C7CF103011F00296E5CFD7
:20FEA000112484E17DCE869580FF06C03196F0930401E093030176CF84910E94067D209107
:20FEC000050230910602E0910301F0910401EECF1F93CF930E94D87CC82F0E94067D0E94D2
:20FEE000D87C182F0E94067DC1362CF0C75511363CF0175508C0C033D4F3C0531136CCF795
:20FF000010330CF01053C295C07FC10F8C2F992787FD9095CF911F910895CF93282F99278F
:20FF200087FD9095807F9070959587959595879595958795959587958A303CF0895AC22F47
:20FF4000CF70CA303CF0C95A06C0805DC22FCF70CA30CCF7C05D0E94067D8C2F0E94067D67
:06FF6000CF910895FFCFD0
:00000001FF
